:1000000095C40000C4C40000C2C40000C0C4000005
:10001000BEC40000BCC40000BAC40000B8C40000E4
:10002000B6C40000B4C40000B2C40000B0C40000F4
:1000300096C60000ACC40000AAC40000A8C400001A
:10004000A6C40000A4C40000A2C40000A0C4000014
:100050009EC400009CC400009AC400000C941E15AD
:1000600096C400000C9444170C941B1790C4000015
:100070008EC400008CC400008AC4000088C4000044
:1000800086C4000084C4000082C4000080C4000054
:100090007EC400007CC400007AC400000C947A176F
:1000A00076C4000074C4000072C4000070C4000074
:1000B0006EC400006CC400006AC4000068C4000084
:1000C00066C4000064C4000062C4000060C4000094
:1000D0005EC400005CC400005AC4000058C40000A4
:1000E00056C4000063146614551459145F149D140B
:1000F0006A146E14741478147C14821486148A148E
:100100009D1490149414981400407A10F35A00A08F
:10011000724E18090010A5D4E80000E876481700D0
:1001200000E40B54020000CA9A3B000000E1F50510
:10013000000080969800000040420F000000A0865A
:1001400001000000102700000000E803000000008C
:100150006400000000000A00000000000100000030
:1001600000002C76D888DC674F0823DFC1DFAE594A
:10017000E1B1B796E5E3E453C63AE651997696E8DD
:10018000E6C28426EB898C9B62ED407C6FFCEFBC61
:100190009C9F40F2BAA56FA5F490055A2AF75C938C
:1001A0006B6CF9676DC11BFCE0E40D47FEF520E6C2
:1001B000B500D0ED902E0300943577050080841EA5
:1001C000080000204E0A000000C80C333333330F00
:1001D000986E12831141EF8D2114893BE65516CF9D
:1001E000FEE6DB18D1844B381BF77C1D901DA4BBA9
:1001F000E424203284725E228100C9F124ECA1E55E
:100200003D27424D5020666F726D6174206E6F7491
:10021000207265636F676E697A65642E004C6F614A
:1002200064656420696E2000496D616765207369AB
:100230007A653A20004269742044657074683A20F7
:10024000004865616465722073697A653A200049E7
:100250006D616765204F66667365743A2000466974
:100260006C652073697A653A200046696C65206E7A
:100270006F7420666F756E64004C6F6164696E67A1
:1002800020696D616765202700000020002300269B
:100290000029002C002F003200000100000301069D
:1002A00001090100000A0B02090C0D0E08070304E6
:1002B000010000000000000000000000000000003D
:1002C000000000000000000000000000000000121C
:1002D00011100000000000000000000000000000FD
:1002E0000000000000000000007C3C3E5E2B3D3F13
:1002F0002F5B5D3B2C2A225C0001021020200808A5
:100300001020401020408002010201080402010177
:100310000204081020408080402010080402018060
:1003200004020180402010080402010804020101B7
:1003300002040810204080010204081020408000C0
:10034000002200250028002B002E0031003400027E
:10035000010000050108010B010505050507050859
:10036000080808020202020A0A0808040404040138
:10037000010101010101010303030303030303045A
:100380000707070C0C0C0C0C0C0C0C0202020206EA
:10039000060606060606060B0B0B0B0B0B0B0B00DB
:1003A000002100240027002A002D00300033000126
:1003B000010000040107010A01EF03038002CF03DB
:1003C00000C130ED0464031281E803850078CB0599
:1003D000392C003402F70120EA020000C00123C1D9
:1003E0000110C5023E28C701863601483701003A90
:1003F0000155B1020018B603088227F20100260158
:1004000001E00F0F312B0C0E084EF1370710030ED1
:100410000900E10F000E1403110731C148080F0C49
:1004200031360F118029800000000000003E5B4F34
:100430005B3E3E6B4F6B3E1C3E7C3E1C183C7E3C44
:10044000181C577D571C1C5E7F5E1C00183C180052
:10045000FFE7C3E7FF0018241800FFE7DBE7FF30E2
:10046000483A060E2629792926407F050507407F50
:1004700005253F5A3CE73C5A7F3E1C1C08081C1CC3
:100480003E7F14227F22145F5F005F5F06097F01B9
:100490007F006689956A606060606094A2FFA294A4
:1004A00008047E040810207E201008082A1C080872
:1004B0001C2A08081E101010100C1E0C1E0C3038C0
:1004C0003E3830060E3E0E06000000000000005FC1
:1004D00000000007000700147F147F14242A7F2ADD
:1004E000122313086462364956205000080703009F
:1004F000001C2241000041221C002A1C7F1C2A08EB
:10050000083E08080080703000080808080800004D
:1005100060600020100804023E5149453E00427FC1
:10052000400072494949462141494D331814127F10
:100530001027454545393C4A4949314121110907B0
:100540003649494936464949291E00001400000031
:100550004034000000081422411414141414004103
:1005600022140802015909063E415D594E7C1211C0
:10057000127C7F494949363E414141227F414141F8
:100580003E7F494949417F090909013E4141517373
:100590007F0808087F00417F41002040413F017FE4
:1005A000081422417F404040407F021C027F7F04AC
:1005B00008107F3E4141413E7F090909063E4151F5
:1005C000215E7F09192946264949493203017F01E5
:1005D000033F4040403F1F2040201F3F4038403FE6
:1005E000631408146303047804036159494D4300FC
:1005F0007F4141410204081020004141417F040233
:1006000001020440404040400003070800205454C9
:1006100078407F28444438384444442838444428A7
:100620007F385454541800087E090218A4A49C78FA
:100630007F0804047800447D40002040403D007F56
:100640001028440000417F40007C047804787C0836
:100650000404783844444438FC182424181824240A
:1006600018FC7C08040408485454542404043F44EF
:10067000243C4040207C1C2040201C3C4030403C1E
:1006800044281028444C9090907C4464544C44007E
:1006900008364100000077000000413608000201E2
:1006A0000204023C2623263C1EA1A161123A4040CE
:1006B000207A38545455592155557941225454784B
:1006C00042215554784020545579400C1E527212E4
:1006D000395555555939545454593955545458006D
:1006E00000457C410002457D420001457C407D1271
:1006F00011127DF0282528F07C54554500205454D3
:100700007C547C0A097F4932494949323A4444447D
:100710003A324A4848303A4141217A3A42402078B8
:10072000009DA0A07D3D4242423D3D4040403D3CB9
:1007300024FF2424487E4943662B2FFC2F2BFF09DE
:1007400029F620C0887E09032054547941000044D2
:100750007D413048484A32384040227A007A0A0ABD
:10076000727D0D19317D2629292F28262929292630
:1007700030484D4020380808080808080808382F75
:1007800010C8ACBA2F102834FA00007B00000814FF
:100790002A142222142A14085500550055AA55AAD5
:1007A00055AAFF55FF55FF000000FF00101010FF75
:1007B00000141414FF001010FF00FF1010F010F0D0
:1007C000141414FC001414F700FF0000FF00FF14C1
:1007D00014F404FC141417101F10101F101F14140D
:1007E000141F00101010F0000000001F1010101057
:1007F0001F10101010F010000000FF10101010104B
:1008000010101010FF10000000FF140000FF00FF88
:1008100000001F10170000FC04F414141710171424
:1008200014F404F40000FF00F71414141414141446
:10083000F700F7141414171410101F101F141414B9
:10084000F4141010F010F000001F101F0000001F23
:1008500014000000FC140000F010F01010FF10FF56
:10086000141414FF141010101F00000000F010FFEB
:10087000FFFFFFFFF0F0F0F0F0FFFFFF00000000CF
:1008800000FFFF0F0F0F0F0F3844443844FC4A4A53
:100890004A347E02020606027E027E026355494108
:1008A000633844443C04407E201E2006027E02023F
:1008B00099A5E7A5991C2A492A1C4C7201724C3053
:1008C0004A4D4D303048784830BC625A463D3E492A
:1008D0004949007E0101017E2A2A2A2A2A44445FCE
:1008E000444440514A444040444A51400000FF01C2
:1008F00003E080FF000008086B6B083612362436D0
:10090000060F090F06000018180000001010003034
:1009100040FF0101001F01011E00191D1712003CBC
:100920003C3C3C00000000000D34A13611241FBEE9
:10093000CFEFD1E2DEBFCDBF00E00CBF16E0A0E0FC
:10094000B2E0E4E7FCE700E00BBF02C007900D92C5
:10095000A43CB107D9F72BE0A4ECB6E001C01D928E
:10096000A830B207E1F714E0C5E9D4E000E006C022
:1009700021970109802FFE010E94B13BC439D107A4
:1009800080E00807A9F70E94AB350C94293E38CBCC
:10099000089580E090E008958F929F92AF92BF9269
:1009A000CF92DF92EF92FF92CF93DF9300D000D0EF
:1009B000CDB7DEB78091C7068823C9F181E09AE000
:1009C0000E940B246B017C0181E09AE00E94C80E1A
:1009D0009C01A4E6B0E00E94C13A2FEF33E040E072
:1009E00050E00E94793A49015A01213737414105C7
:1009F0005105DCF020E030E040E85FE3C701B601DC
:100A00000E94603987FF11C01092C70668EB72E040
:100A1000CE0101960E94A016CE0101960E943330AD
:100A2000CE0101960E94821636C0A40130C066E352
:100A300081E09AE00E946912882369F10E943232B3
:100A400081E08093C7066AED72E0CE0101960E94B4
:100A5000A016CE0101960E943330CE0101960E946D
:100A6000821681E09AE00E940B246B017C0181E0F8
:100A70009AE00E94C80E9C01A4E6B0E00E94C13A30
:100A80002FEF33E040E050E00E94793AA901C7011E
:100A9000B6010E9499338091C6068823C9F188EF78
:100AA00099E00E940B246B017C0188EF99E00E9481
:100AB000C80E9C01A4E6B0E00E94C13A2FEF33E0DB
:100AC00040E050E00E94793A49015A01213737410C
:100AD00041055105DCF020E030E040E85FE3C7016C
:100AE000B6010E94603987FF11C01092C6066CEFF4
:100AF00072E0CE0101960E94A016CE0101960E94DE
:100B00003330CE0101960E94821636C0A40130C057
:100B100067E388EF99E00E946912882369F10E94D7
:100B2000323281E08093C6066EE173E0CE01019619
:100B30000E94A016CE0101960E943330CE0101968C
:100B40000E94821688EF99E00E940B246B017C01C1
:100B500088EF99E00E94C80E9C01A4E6B0E00E94D4
:100B6000C13A2FEF33E040E050E00E94793AA9010A
:100B7000C701B6010E9425338091C5068823C9F1BB
:100B80008FEE99E00E940B246B017C018FEE99E0BF
:100B90000E94C80E9C01A4E6B0E00E94C13A2FEF6B
:100BA00033E040E050E00E94793A49015A01213790
:100BB000374141055105DCF020E030E040E85FE3DB
:100BC000C701B6010E94603987FF11C01092C506A7
:100BD00060E473E0CE0101960E94A016CE0101965A
:100BE0000E943330CE0101960E94821636C0A401C5
:100BF00030C068E38FEE99E00E946912882369F1A2
:100C00000E94323281E08093C50662E673E0CE0135
:100C100001960E94A016CE0101960E943330CE01AB
:100C200001960E9482168FEE99E00E940B246B01C0
:100C30007C018FEE99E00E94C80E9C01A4E6B0E012
:100C40000E94C13A2FEF33E040E050E00E94793A31
:100C5000A901C701B6010E94B0328091C406882361
:100C6000C9F186EE99E00E940B246B017C0186EEAF
:100C700099E00E94C80E9C01A4E6B0E00E94C13A2F
:100C80002FEF33E040E050E00E94793A49015A01E9
:100C90002137374141055105DCF020E030E040E8E4
:100CA0005FE3C701B6010E94603987FF11C010924F
:100CB000C40664E873E0CE0101960E94A016CE013E
:100CC00001960E943330CE0101960E94821636C0F2
:100CD000A40130C069E386EE99E00E94691288237E
:100CE00069F10E94323281E08093C40666EA73E0C3
:100CF000CE0101960E94A016CE0101960E943330CB
:100D0000CE0101960E94821686EE99E00E940B2485
:100D10006B017C0186EE99E00E94C80E9C01A4E65E
:100D2000B0E00E94C13A2FEF33E040E050E00E9473
:100D3000793AA901C701B6010E943A3226960FB648
:100D4000F894DEBF0FBECDBFDF91CF91FF90EF9043
:100D5000DF90CF90BF90AF909F908F9008951F929B
:100D60000F920FB60F9211248F930FB6F894A89597
:100D700080916000886180936000109260000FBED7
:100D80008F910F900FBE0F901F9018951F93CF93C8
:100D9000DF93262FFC0133A137FF09C07EBD0DB4C0
:100DA00007FEFDCF2EBD0DB407FEFDCF0CC0672F93
:100DB000122FEC010E94D51D612FCE01DF91CF9142
:100DC0001F910C94D51DDF91CF911F9108952F9203
:100DD0003F924F925F926F927F928F929F92AF92CB
:100DE000BF92CF92DF92EF92FF920F931F93CF9318
:100DF000DF93CDB7DEB7C557D1400FB6F894DEBF4D
:100E00000FBECDBFE091E208F091E30882E080835D
:100E1000E091DE08F091DF081082E091E008F091A7
:100E2000E1088FEC80831092EA08E091E608F091E7
:100E3000E70886E08083E091E408F091E50880818E
:100E400080618083E091E408F091E508808188600A
:100E50008083E091E408F091E508808180688083D8
:100E6000E091E408F091E50880818F7D808340E087
:100E700050E0BA018AE09AE00E94C01F61E08AE077
:100E80009AE00E94761F8091A009882321F08BE9C7
:100E900099E00E94A61A10927C0910927A09109289
:100EA00077091092760983E1809375090E941215E3
:100EB0006B017C0161E0809175090E949E1461E0E4
:100EC000809175090E943A120E94932F82E58093C7
:100ED0006F091092700980916F09909170090E94BA
:100EE000902F2AE0CF59DE4F2883C156D1408FEF93
:100EF0000E94D91BCF59DE4F3881C156D1403150A5
:100F0000CF59DE4F3883C156D1403111F0CF860121
:100F10000E948F2F81E799E00E94B51B20E030E00E
:100F2000A90160E081E799E00E94121CF82E8093ED
:100F30007B0951E0851749F00E941215601B710B67
:100F4000613D774058F381E056C02AEA31E040E045
:100F500050E068E081E799E00E94121C82FF03C024
:100F6000F0927C0910C044E0F42E0E94E01B8093B4
:100F70007B09FA94F110F9CF8A3A11F082E03BC074
:100F800082E080937C0980917C09823021F0C12C21
:100F9000D12C760105C0C12CD12CE12C30E4F32EEC
:100FA00020E030E0A90167E381E799E00E94121C8C
:100FB000A701960169E281E799E00E94121C8093E3
:100FC0007B09882349F00E941215601B710B613D5B
:100FD000774030F388E00FC080917C09823001F5C2
:100FE00020E030E0A9016AE381E799E00E94121C49
:100FF000882341F086E08093760981E799E00E949A
:10100000CB1B6EC30E94E01B807C803C19F483E004
:1010100080937C090E94E01B0E94E01B0E94E01B61
:1010200081E799E00E94CB1B80E580936F091092C5
:10103000700981E00E94E310882341F08BE999E078
:101040000E948F10882309F44BC307C080E00E94E0
:10105000E310882309F444C3F1CF6FEF7FEF8AE0F8
:101060009AE00E94BD2DC85BDE4F19821882C854D9
:10107000D14088EE93E0A0E0B0E0C65BDE4F88830D
:101080009983AA83BB83CA54D14082EA92E0CA5BA7
:10109000DE4F99838883C654D140C15ADE4F1982EE
:1010A0001882CF55D140CE5ADE4F1882C255D1405A
:1010B0000E941215C259DE4F688379838A839B830D
:1010C000CE56D1408091120A9091130A1816190633
:1010D0000CF001C18091140A9091150A1816190696
:1010E0000CF0F9C0B8D689E792E0BAD668EC73E0A4
:1010F00082ED98E00E94061787E215D7ACD61C82D5
:101100001B8206E412E01A8309831E82CE01019637
:101110000E948F108B819C81C05FDE4F99838883F2
:10112000C051D140C25FDE4F19830883CE50D140F9
:101130008D81CE5EDE4F8883C251D1408E81CD5EDF
:10114000DE4F8883C351D1404F81588569857A85A8
:10115000CC5EDE4F488359836A837B83C451D14080
:101160004B855C856D857E85C85EDE4F48835983DF
:101170006A837B83C851D1404F85588969897A89B0
:10118000C45EDE4F488359836A837B83CC51D14050
:101190009B89C05EDE4F9883C052D1404C895D89E7
:1011A0006E897F89CF5DDE4F488359836A837B8355
:1011B000C152D140488D598D6A8D7B8DCB5DDE4FFC
:1011C000488359836A837B83C552D1402C8D3D8DE2
:1011D000C75DDE4F39832883C952D140CD50DF4FE0
:1011E00019821882C35FD040CF50DF4F1983088324
:1011F000C15FD040CA50DF4F1882C65FD040811116
:1012000071C2C35DDE4F19821882CD52D14088EE83
:1012100093E0A0E0B0E0C15DDE4F88839983AA83AC
:10122000BB83CF52D140CC5BDE4F19821882C454AD
:10123000D140C95CDE4F1882C753D140C35DDE4F39
:1012400088819981CD52D140C85BDE4F99838883D4
:10125000C854D140C15DDE4F88819981AA81BB818C
:10126000CF52D140C65BDE4F88839983AA83BB836C
:10127000CA54D140CD5CDE4F88819981AA81BB815F
:10128000C353D140C25BDE4F88839983AA83BB835B
:10129000CE54D1408DE0EBE2F1E0EC0FFD1F3C9627
:1012A000A6E4B1E0AC0FBD1F1C9601900D928A958B
:1012B000E1F7CC5BDE4FE881F981C454D140C15ADB
:1012C000DE4FF983E883CF55D140309709F086C2CD
:1012D0008AE692E0C5D560EA7FE080E090E00E9477
:1012E000DA1411E06FEF7FEF8AE09AE00E94BD2DE3
:1012F00064ED73E0CE0101960E94A016CE01019626
:101300000E943330CE0101960E9482166AEF70E08F
:1013100080E090E00E94DA1411110EC06EEE73E0CE
:10132000CE0101960E94A016CE0101960E94333094
:10133000CE0101960E9482166DE074E0CE01019606
:101340000E94A016CE0101960E943330CE01019674
:101350000E94821661E0CF59DE4F8881C156D1408C
:101360000E949E1460E0CF59DE4F8881C156D14063
:101370000E943A12CF59DE4F3881C156D1403F5FAB
:10138000CF59DE4F3883C156D140343119F710E2BE
:1013900061E0812F0E949E1460E0812F0E943A122A
:1013A0001F5F1633A9F763E474E0CE0101960E9433
:1013B000A016CE0101960E943330CE0101960E9404
:1013C000821682ED98E00E94C613E091E408F09145
:1013D000E50880818F7E8083E091E408F091E50844
:1013E0008081877F8083E091E408F091E508808127
:1013F0008F778083E091E408F091E50880818F7D0C
:1014000080838091EC088093EB0880916400816078
:101410008093640080916400826080936400809176
:101420006500816080936500809165008260809393
:1014300065008091640088608093640080916400FE
:10144000806480936400809165008860809365006B
:101450008091650080618093650080916500806265
:101460008093650069E674E0CE0101960E94A016A3
:10147000CE0101960E943330CE0101960E94821661
:1014800010927A0011E010938C0A6FE874E0CE019C
:1014900001960E94A016CE0101960E943330CE0123
:1014A00001960E94821610938B0A66E381E09AE00F
:1014B0000E946912811111C068EB72E0CE010196A1
:1014C0000E94A016CE0101960E943330CE010196F3
:1014D0000E9482161092C70628C060EE74E0CE010A
:1014E00001960E94A01681E09AE00E94412460E1EA
:1014F00070E0CE0101960E941416BE016F5F7F4F0F
:10150000CE018F509F4F0E948716CE018F509F4F64
:101510000E943330CE018F509F4F0E94821610934D
:10152000C706CE0101960E94821667E388EF99E014
:10153000D0D7811111C06CEF72E0CE0101960E94EC
:10154000A016CE0101960E943330CE0101960E9472
:1015500082161092C60629C06CE075E0CE01019695
:101560000E94A01688EF99E00E94412460E170E09B
:10157000CE0101960E941416BE016F5F7F4FCE010F
:101580008F509F4F0E948716CE018F509F4F0E9411
:101590003330CE018F509F4F0E94821681E080939E
:1015A000C606CE0101960E94821668E38FEE99E08E
:1015B00090D7811111C060E473E0CE0101960E94C2
:1015C000A016CE0101960E943330CE0101960E94F2
:1015D00082161092C50629C068E375E0CE01019617
:1015E0000E94A0168FEE99E00E94412460E170E015
:1015F000CE0101960E941416BE016F5F7F4FCE018F
:101600008F509F4F0E948716CE018F509F4F0E9490
:101610003330CE018F509F4F0E94821681E080931D
:10162000C506CE0101960E94821669E386EE99E016
:1016300050D7811111C064E873E0CE0101960E9479
:10164000A016CE0101960E943330CE0101960E9471
:1016500082161092C40629C064E675E0CE01019698
:101660000E94A01686EE99E00E94412460E170E09D
:10167000CE0101960E941416BE016F5F7F4FCE010E
:101680008F509F4F0E948716CE018F509F4F0E9410
:101690003330CE018F509F4F0E94821681E080939D
:1016A000C406CE0101960E94821676D9CB58DE4F31
:1016B0000FB6F894DEBF0FBECDBFDF91CF911F9163
:1016C0000F91FF90EF90DF90CF90BF90AF909F90E1
:1016D0008F907F906F905F904F903F902F900895E4
:1016E00010E000CE48EC53E0BE01625F7E4FCE01B9
:1016F0008F509F4F2ED4882309F483CDCE01825F73
:101700009E4F0E94A61ACD50DF4F88819981C35FFA
:10171000D0409C838B831A830983CB50DF4F888111
:10172000C55FD0408D83CA50DF4F8881C65FD040EF
:101730008E83C950DF4F88819981AA81BB81C75FA1
:10174000D0408F839887A987BA87C550DF4F88819B
:101750009981AA81BB81CB5FD0408B879C87AD8765
:10176000BE87C150DF4F88819981AA81BB81CF5F3D
:10177000D0408F87988BA98BBA8BCD5FDE4F888145
:10178000C350D1408B8BCC5FDE4F88819981AA8179
:10179000BB81C450D1408C8B9D8BAE8BBF8BC85FFF
:1017A000DE4F88819981AA81BB81C850D140888F42
:1017B000998FAA8FBB8FC45FDE4F88819981CC50EF
:1017C000D1409D8F8C8F48EC53E0BE016F5F7F4FFF
:1017D000CE01855D9E4F0E94571D30CD85818823A7
:1017E00009F476CDCE018A5B9E4F7CD282349D4433
:1017F00009F020C28EE592E033D3CE018A5B9E4F82
:101800008AD29CD3CE018A5B9E4F85D2CE018A5B61
:101810009E4F81D26B017C018FE492E021D3C701FE
:10182000B6018CD381E492E01BD3CE018A5B9E4F3C
:1018300072D284D3CE018A5B9E4F6DD22B013C01C4
:10184000CE018A5B9E4F67D2CE59DE4F6883798383
:101850008A839B83C256D140CE018A5B9E4F42D27F
:10186000019709F0E7C1CE018A5B9E4F3BD2182F4A
:1018700085E392E0F5D2612F70E080E090E04AE0ED
:1018800010D3E9D2183109F0D5C1CE018A5B9E4F41
:1018900042D2CA59DE4F688379838A839B83C656B6
:1018A000D140672B682B692B09F0C4C188E292E014
:1018B000D7D24201052C000CAA08BB08B7FE0BC00A
:1018C0008DE231D366277727CB01681979098A0918
:1018D0009B094AE003C04AE0C501B401E2D2CE59F7
:1018E000DE4F08811981C256D14088E71CD3CE59FA
:1018F000DE4F28813981C256D1404901330FAA08F1
:10190000BB08B7FE0BC08DE20ED366277727CB014D
:10191000681979098A099B094AE003C04AE0C501B0
:10192000B401BFD298D252013FEFA31AB30AC50146
:10193000880F991FA80EB91E4CEFA422B5010B2CDD
:10194000000C880B990BC659DE4F688379838A8314
:101950009B83CA56D14017FF0FC0CE59DE4F088176
:101960001981C256D140119501951109CE59DE4F0A
:101970001882C256D14006C071E0CE59DE4F78833E
:10198000C256D140C20101974801A1E08A1A9108CC
:1019900097FD17C1BFEF8B169B0609F412C120906B
:1019A000120A3090130A821593050CF4120160900C
:1019B000140A7090150A861497040CF438018AE012
:1019C0009AE00E946E1A8301910140E050E060E0CD
:1019D00070E08AE09AE00E94AB1E9401D5010E945B
:1019E000B93B4B015C018C0C9D1CAE1CBF1C412CF7
:1019F000512C20EF461457040CF0DFC0CE59DE4FB7
:101A00003881C256D140332369F0CA59DE4F48812C
:101A100059816A817B81C656D140480D591D6A1D86
:101A20007B1D02C0B701A601C15ADE4FE881F981D2
:101A3000CF55D140309729F082859385A485B5850F
:101A400003C08FEF9FEFDC0184179507A607B70748
:101A5000D9F18AE09AE0CE58DE4F4883C257D14090
:101A6000CD58DE4F5883C357D140CC58DE4F6883E2
:101A7000C457D140CB58DE4F7883C557D1400E9420
:101A8000C419C15ADE4F88819981CF55D140CE58B3
:101A9000DE4F4881C257D140CD58DE4F5881C357E1
:101AA000D140CC58DE4F6881C457D140CB58DE4F6F
:101AB0007881C557D140009711F00E94B5268AE081
:101AC0009AE00E946E1A20EF00E010E00215130564
:101AD0000CF04FC0203FC0F08AE09AE00E94C41989
:101AE000C15ADE4F88819981CF55D140009739F096
:101AF00040EF50E0BE016F5F7F4F0E94E5288AE013
:101B00009AE00E946E1A20E0E1E0F0E0EC0FFD1F89
:101B1000E20FF11D808191E0920FE1E0F0E0EC0F27
:101B2000FD1FE90FF11D608192E0920FE1E0F0E00E
:101B3000EC0FFD1FE90FF11D2D5F9081987F6C7FE9
:101B400048E0649FB0011124792B8695869586958F
:101B5000682B8AE09AE0CE58DE4F2883C257D140E6
:101B600015D90F5F1F4FCE58DE4F2881C257D14085
:101B7000ADCF5FEF451A550ACA59DE4F888199816A
:101B8000AA81BB81C656D140C659DE4F48815981D2
:101B90006A817B81CA56D140841B950BA60BB70B7B
:101BA000CA59DE4F88839983AA83BB83C656D14026
:101BB000C40ED51EE61EF71E1DCF8AE09AE00E94D5
:101BC000C4198DE192E04CD12DD7C259DE4F288146
:101BD00039814A815B81CE56D140621B730B840BE5
:101BE000950B4AE05ED160ED73E082ED98E00E94D3
:101BF000061731D111E0C15ADE4F88819981CF5546
:101C0000D140009781F00E94A61AC15ADE4F888108
:101C10009981CF55D1400E945A3CC15ADE4F19825A
:101C20001882CF55D140111156CB82E092E018D1E5
:101C300012D151CB10E0DFCFCF93DF93EC016A8B51
:101C40008091000290910102A0910202B0910302E2
:101C50008E879F87A88BB98B80E2689FF001112443
:101C6000E553F94F4489558960E070E0BA01552782
:101C700044274F8B588F698F7A8F828D938DA0E088
:101C8000B0E0482B592B6A2B7B2B4F8B588F698FD9
:101C90007A8F8385887151F4848D958DA68DB78D4B
:101CA0008B8B9C8BAD8BBE8B81E00EC0803111F095
:101CB00080E015C09E012D5E3F4F8B8D9C8D0E9454
:101CC00011268823A9F384E08D8381E08C831E8212
:101CD0001F82188619861A861B861C861D86DF9130
:101CE000CF9108950F931F93CF93DF931F921F926D
:101CF000CDB7DEB78C010E94A31D8983C8010E9465
:101D0000A31D8A8389819A810F900F90DF91CF91D3
:101D10001F910F9108950F931F93CF93DF9300D0DE
:101D20001F92CDB7DEB78C010E94A31D8983C80125
:101D30000E94A31D8A83C8010E94A31D8B83C80132
:101D40000E94A31D8C8369817A818B819C810F9075
:101D50000F900F900F90DF91CF911F910F910895E9
:101D6000FC0144815581608171818CEC99E0CFC682
:101D7000CF93DF93EC0141E050E068EC75E0C7D60B
:101D8000811102C0CE018DD7CE01DF91CF91089590
:101D9000EF92FF920F931F93CF93DF931F921F92A7
:101DA000CDB7DEB728EEE22E23E0F22E02E09E0150
:101DB0002F5F3F4F40E16FE00E94B722098110E0A2
:101DC000102F00278A81082B61E070E080E090E00E
:101DD000F1D5C8010F900F90DF91CF911F910F9116
:101DE000FF90EF9008950F931F931CD66093DA082D
:101DF0007093DB088093DC089093DD08E091D208B3
:101E0000F091D3080284F385E02D82ED98E01995D6
:101E100097FF1EC007D60091DA081091DB082091C9
:101E2000DC083091DD08DC01CB01801B910BA20B9B
:101E3000B30B0091D6081091D7082091D8083091A3
:101E4000D90880179107A207B307C0F28FEF9FEF61
:101E50001F910F91089560E975E082ED98E0D6C773
:101E60000F931F93CF93DF938C01C0E0D0E0F80174
:101E7000EC0FFD1F6491662371F0E091D208F091A0
:101E8000D3080190F081E02D82ED98E01995892B1F
:101E900011F02196ECCFCE01DF91CF911F910F91E0
:101EA00008958F929F92AF92BF920F931F93CF93FB
:101EB000DF93CDB7DEB7A1970FB6F894DEBF0FBEA4
:101EC000CDBF19A2423008F44AE08E010F5D1F4FCA
:101ED000842E912CA12CB12CA50194010E949F3A33
:101EE000E62FB901CA0101501109EA3014F4E05D8E
:101EF00001C0E95CD801EC93232B242B252B61F73F
:101F0000B80182ED98E082D7A1960FB6F894DEBFB3
:101F10000FBECDBFDF91CF911F910F91BF90AF90BA
:101F20009F908F900895E091D208F091D30801908E
:101F3000F081E02D682F82ED98E01994CF93DF9324
:101F40004AE0AFDFEC0187DF8C0F9D1FDF91CF915F
:101F50000895AF92BF92CF92DF92EF92FF920F93CC
:101F60001F93CF93DF93CDB7DEB72B970FB6F894BF
:101F7000DEBF0FBECDBF7C01CE0101966C01FC011E
:101F800090E28BE08C0D91938E13FDCFDA0120E06F
:101F900037E09D91992339F19E3219F0E9EEF2E094
:101FA0000AC03A3009F4A9C028E03AE0F2CF3196ED
:101FB000891709F4A2C084918111F9CF321708F46E
:101FC0009CC08FED890F8E3508F097C081E0820F9D
:101FD000F601E20FF11D2FE9290F2A3108F4905282
:101FE0009083282FD6CF8981803209F486C08B0157
:101FF000FB01838D948DF701948F838FFB011682F3
:102000001782108611861286138614861586A12CD7
:10201000F80182859385A485B585438954896589AE
:10202000768984179507A607B70708F066C025E0EC
:10203000B695A795979587952A95D1F7F82FFF70B4
:10204000BF2EF8018581823008F457C0C8010E9474
:102050008C1D97FD52C0F80182859385A485B585B6
:102060004F96A11DB11D82879387A487B587F0E2A3
:10207000BF9EC0011124BC016553794F61157105E4
:10208000E1F1FB0120812223B1F1253ED9F04BE0A3
:1020900050E0C6010E94DA3D892B09F0B9CF6B2DC3
:1020A000C7012B960FB6F894DEBF0FBECDBFDF91F0
:1020B000CF911F910F91FF90EF90DF90CF90BF9045
:1020C000AF90BACDA11014C0F701B28A40910002BE
:1020D0005091010260910202709103024687578776
:1020E000608B718BFC01E553F94F8081882329F0C7
:1020F000AA24A3948DCFAA2039F380E02B960FB6A3
:10210000F894DEBF0FBECDBFDF91CF911F910F912D
:10211000FF90EF90DF90CF90BF90AF900895CF9356
:10212000DF93FC012581222311F080E049C0EC01FE
:10213000809194098031C1F482E08583178A108EE2
:10214000118E128E8091950990919609A0E0B0E0D1
:1021500025E0880F991FAA1FBB1F2A95D1F7838BF3
:10216000948BA58BB68B19C08032F9F683E08583FA
:1021700040919709509198096091990970919A0935
:10218000478B508F618F728F9F012D5E3F4F8DE780
:1021900099E00E941126882341F28DE799E09C8FF7
:1021A0008B8F81E08C831E821F82188619861A8687
:1021B0001B861C861D861E861F86188A198A1A8A07
:1021C000DF91CF9108958F929F92AF92BF92CF925D
:1021D000DF92EF92FF92CF93DF93C82F81E799E0D0
:1021E0009093C9068093C806CC2369F1C53010F0DE
:1021F00080E00DC140E060E070E0CB010E94A724C8
:102200008823B1F320E1C29FC00111248554994F66
:10221000FC01E254FE4F20812F7751F73C9640811C
:10222000518162817381443651056105710500F366
:102230003497C080D180E280F380C114D104E104DE
:10224000F10421F4D5CFC12CD12C760140E0C70197
:10225000B6010E94A724882359F28091D606909156
:10226000D7068115924021F6A091DB06AA2309F436
:10227000BFCF6091D9067091DA066115710509F436
:10228000B7CF2091D806222309F4B2CFA0938F09AB
:102290002093810980E030E0E1E0F0E0C82FAF0159
:1022A000082E02C0440F551F0A94E2F72417350781
:1022B00041F0982F8F5F983089F789E080938A09E1
:1022C00097CF80938A092091E1063091E20621158B
:1022D000310519F040E050E008C02091EF06309140
:1022E000F0064091F1065091F20620938209309356
:1022F0008309409384095093850946015701860E4E
:10230000971EA11CB11C8092900990929109A092F5
:102310009209B0929309E091DC06F091DD06F0930A
:102320009609E0939509B0E00E94953A860E971EB3
:10233000A81EB91E8092970990929809A0929909B7
:10234000B0929A0985E0EE0FFF1F8A95E1F7E15000
:10235000FE4FEF2FFF27E6958E0E9F1EA11CB11C8E
:1023600080928B0990928C09A0928D09B0928E096F
:102370002091DE063091DF062115310521F0A901FB
:1023800060E070E008C04091EB065091EC0660916F
:10239000ED067091EE06D701C60188199909AA09C0
:1023A000BB09840F951FA61FB71F04C0B695A7953C
:1023B00097958795CA95D2F7809386099093870958
:1023C000A0938809B0938909853F2FE09207A10562
:1023D000B10510F48CE018C0853F9F4FA105B105F1
:1023E00010F480E111C08091F7069091F806A09159
:1023F000F906B091FA068093970990939809A093F3
:102400009909B0939A0980E28093940981E0DF9161
:10241000CF91FF90EF90DF90CF90BF90AF909F90C3
:102420008F900895CF93DF93282F30E0F901ED5579
:10243000FD4F8491F901E750FD4FD491F901E75A1E
:10244000FC4FC491CC2389F0811122D2EC2FF0E013
:10245000EE0FFF1FE757FD4FA591B491EC91ED23CF
:1024600081E090E021F480E002C080E090E0DF9124
:10247000CF9108951F93CF93DF93282F30E0F90178
:10248000ED55FD4F8491F901E750FD4FD491F901CD
:10249000E75AFC4FC491CC23C1F0162F8111F8D11B
:1024A000EC2FF0E0EE0FFF1FE15CFC4FA591B49123
:1024B0008FB7F894111105C09C91ED2FE095E92399
:1024C00002C0EC91ED2BEC938FBFDF91CF911F9168
:1024D0000895CF92DF92EF92FF920F931F93CF93C5
:1024E000DF931F921F92CDB7DEB76C01FC016483AE
:1024F0001FEF17831092D1081092D0081092CF08C6
:102500001092CE081092CD0881E08093CC081092F2
:10251000CB0861E084E1AEDF61E085E1ABDF809173
:10252000B9008E7F8093B9008091B9008D7F809330
:10253000B90088E48093B80085E48093BC001A83D6
:1025400001E09E012E5F3F4F4FE760E0C6010E9411
:10255000B62164EF71E080E090E02CD28DE7E82EA8
:10256000F12C9E012F5F3F4F41E060E0C6010E94C9
:10257000B722998181E0953509F080E00F900F90A6
:10258000DF91CF911F910F91FF90EF90DF90CF904F
:1025900008953FB7F8948091B80A9091B90AA09134
:1025A000BA0AB091BB0A26B5A89B05C02F3F19F007
:1025B0000196A11DB11D3FBFBA2FA92F982F8827C3
:1025C000820F911DA11DB11DBC01CD0142E0660F1E
:1025D000771F881F991F4A95D1F70895CF92DF92F0
:1025E000EF92FF920F931F93CF93DF936C017A01C9
:1025F0008B01C0E0D0E0CE15DF0589F0D8016D91E8
:102600008D01D601ED91FC910190F081E02DC60184
:102610001995892B11F47E0102C02196ECCFC701D8
:10262000DF91CF911F910F91FF90EF90DF90CF90AE
:102630000895FC01538D448D252F30E0842F90E0C8
:10264000821B930B541710F0CF96089501970895AD
:10265000FC01918D828D981761F0828DDF01A80FAA
:10266000B11D5D968C91928D9F5F9F73928F90E0CC
:1026700008958FEF9FEF0895FC01918D828D98173B
:1026800031F0828DE80FF11D858D90E008958FEF78
:102690009FEF0895FC01918D228D892F90E0805C41
:1026A0009F4F821B91098F739927089582ED98E0BF
:1026B000F1DF21E0892B09F420E0822F0895FC014D
:1026C000848DDF01A80FB11DA35ABF4F2C91848DBB
:1026D00090E001968F739927848FA689B7892C93F0
:1026E000A089B1898C9180648C93938D848D98138B
:1026F00006C00288F389E02D80818F7D8083089554
:10270000EF92FF920F931F93CF93DF93EC0181E041
:10271000888F9B8D8C8D981305C0E889F9898081FD
:1027200085FD23C0F62E0B8D10E00F5F1F4F0F733A
:102730001127E02E8C8DE8120BC00FB607FCFACFE4
:10274000E889F989808185FFF5CFCE01B8DFF2CF26
:102750008B8DFE01E80FF11DE35AFF4FF0820B8FC6
:10276000EA89FB898081806207C0EE89FF896083E6
:10277000E889F98980818064808381E090E0DF913D
:10278000CF911F910F91FF90EF900895CF93DF931A
:10279000EC01888D8823C1F0EA89FB89808185FD61
:1027A00005C0A889B9898C9186FD0EC00FB607FCBB
:1027B000F5CF808185FFF2CFA889B9898C9185FFFB
:1027C000EDCFCE017CDFE8CFDF91CF91089580E09F
:1027D00090E0892B19F06ADF811125C080E090E03C
:1027E000892B41F080E090E0892B21F00E940000CD
:1027F00081111CC080E090E0892B41F080E090E0E6
:10280000892B21F00E940000811113C080E090E02C
:10281000892BA1F080E090E0892B81F00E940000DC
:1028200081110AC008950E940000D8CF0E940000C4
:10283000E1CF0E940000EACF0C94000008950E94AE
:10284000D63D0F931F93CF93DF93EC01888199813D
:10285000009729F02A813B812617370788F48B01DE
:102860006F5F7F4F0E94F23C009761F099838883ED
:102870001B830A832C813D81232B11F4FC011082E0
:1028800081E001C080E0DF91CF911F910F91089509
:1028900090E0FC013197E231F10508F04EC0882745
:1028A000EE58FF4F8F4F0C94B13B809180008F7793
:1028B00003C0809180008F7D809380000895809177
:1028C0008000877FF9CF84B58F7702C084B58F7D74
:1028D00084BD08958091B0008F7703C08091B000CF
:1028E0008F7D8093B0000895809190008F7707C00E
:1028F000809190008F7D03C080919000877F8093AE
:10290000900008958091A0008F7707C08091A0006B
:102910008F7D03C08091A000877F8093A0000895E1
:10292000809120018F7707C0809120018F7D03C0A7
:1029300080912001877F809320010895CF93DF93BA
:1029400090E0FC01E750FD4F2491FC01E75AFC4F59
:102950008491882361F190E0880F991FFC01E15672
:10296000FC4FC591D491FC01E15CFC4FA591B49161
:10297000611109C09FB7F8948881209582238883CC
:10298000EC912E230BC0623061F49FB7F89438812C
:10299000822F809583238883EC912E2B2C939FBFCD
:1029A00006C08FB7F894E8812E2B28838FBFDF9164
:1029B000CF9108958F929F92AF92BF92CF92DF9264
:1029C000EF92FF926B017C01E4DD4B015C01C114CD
:1029D000D104E104F104E9F0DCDDDC01CB0188196C
:1029E0009909AA09BB09883E9340A105B10578F36E
:1029F00021E0C21AD108E108F10888EE880E83E0D0
:102A0000981EA11CB11CC114D104E104F10421F7EA
:102A1000DECFFF90EF90DF90CF90BF90AF909F9070
:102A20008F9008952FB7F8946091B40A7091B50A09
:102A30008091B60A9091B70A2FBF08951F920F9206
:102A40000FB60F9211242F933F938F939F93AF93C1
:102A5000BF938091B40A9091B50AA091B60AB09143
:102A6000B70A3091B30A23E0230F2D3720F40196E3
:102A7000A11DB11D05C026E8230F0296A11DB11DA1
:102A80002093B30A8093B40A9093B50AA093B60A30
:102A9000B093B70A8091B80A9091B90AA091BA0A86
:102AA000B091BB0A0196A11DB11D8093B80A909305
:102AB000B90AA093BA0AB093BB0ABF91AF919F9194
:102AC0008F913F912F910F900FBE0F901F901895EF
:102AD000FC0124813581232B31F421E0611571053E
:102AE000A1F0FB0108C0FC01808191816115710595
:102AF00031F421E0FC018081882339F005C00E9477
:102B0000F03D21E0892B09F020E0822F0895EF921B
:102B1000FF920F931F93CF93DF93FC0124813581A4
:102B20006115710511F480E018C041155105A1F03F
:102B30007B01EC018A01020F131FB80182DE88239A
:102B400091F3288139818C819D81B701820F931F78
:102B50000E94F93D1D830C8381E0DF91CF911F918D
:102B60000F91FF90EF900895EF92FF920F931F93B4
:102B7000CF93DF93CDB7DEB764970FB6F894DEBF7F
:102B80000FBECDBF7C01CB01BA018E010F5F1F4F7D
:102B900022E044E00E94A936BC01FC010190002023
:102BA000E9F73197AF01481B590BC701B0DF6496B5
:102BB0000FB6F894DEBF0FBECDBFDF91CF911F914E
:102BC0000F91FF90EF900895EF92FF920F931F9354
:102BD000CF93DF93CDB7DEB764970FB6F894DEBF1F
:102BE0000FBECDBF7C01CB01BA018E010F5F1F4F1D
:102BF00022E044E00E94A936BC01FC0101900020C3
:102C0000E9F73197AF01481B590BC70180DF649684
:102C10000FB6F894DEBF0FBECDBFDF91CF911F91ED
:102C20000F91FF90EF900895EF92FF920F931F93F3
:102C3000CF93DF93CDB7DEB728970FB6F894DEBFFA
:102C40000FBECDBF7C01CB014AE08E010F5F1F4F4D
:102C5000B8010E94C836F80101900020E9F73197C9
:102C6000AF01401B510BB801C70151DF28960FB6C9
:102C7000F894DEBF0FBECDBFDF91CF911F910F91B2
:102C8000FF90EF9008956115710549F0FB010190E7
:102C90000020E9F73197AF01461B570B38CF80E092
:102CA0000895CF93DF93EC0188819981009711F00B
:102CB0000E945A3C198218821D821C821B821A8231
:102CC000DF91CF910895EF92FF920F931F93CF93CF
:102CD000DF93EC017B018A01BA01B3DD811103C0EE
:102CE000CE01DFDF07C01D830C83B7018881998186
:102CF0000E94F93DCE01DF91CF911F910F91FF907E
:102D0000EF900895FC01808191810C945A3CFB0165
:102D1000DC0111961C921E9213961C921E92129721
:102D200015961C921E9214978617970741F06081A2
:102D300071816115710519F044815581C4CF0895E1
:102D4000FC01118210821382128215821482611595
:102D5000710549F0FB0101900020E9F73197AF01BF
:102D6000461B570BB0CF0895BF92CF92DF92EF92E0
:102D7000FF920F931F93CF93DF937C016B01EA01C6
:102D800089012417350720F48D2FE901042F182F0E
:102D900062E975E0C701D4DFD60114968D919C914C
:102DA0001597C817D90738F58017910708F48C01D3
:102DB000D601ED91FC911197E00FF11FB0801082C8
:102DC0004D915C91BA016C0F7D1F6115710559F031
:102DD000FB0101900020E9F73197AF01461B570B2B
:102DE000C70171DF02C0C7015CDFD601ED91FC9124
:102DF000E00FF11FB082C701DF91CF911F910F91BA
:102E0000FF90EF90DF90CF90BF900895611571050E
:102E100079F0FB0101900020E9F73197AF01461BE3
:102E2000570BDC01ED91FC910280F381E02D1994A8
:102E300080E090E008951F920F920FB60F92112438
:102E40000BB60F922F933F934F935F936F937F93A4
:102E50008F939F93AF93BF93EF93FF9382ED98E08F
:102E60002EDCFF91EF91BF91AF919F918F917F9158
:102E70006F915F914F913F912F910F900BBE0F90EB
:102E80000FBE0F901F9018951F920F920FB60F92C2
:102E900011240BB60F922F938F939F93EF93FF9371
:102EA000E091E208F091E3088081E091E808F09178
:102EB000E90882FD12C090818091EB088F5F8F73CB
:102EC0002091EC08821751F0E091EB08F0E0EE520F
:102ED000F74F958F8093EB0801C08081FF91EF91B0
:102EE0009F918F912F910F900BBE0F900FBE0F905F
:102EF0001F9018951F920F920FB60F9211240BB6C8
:102F00000F922F933F934F935F936F937F938F9382
:102F10009F93AF93BF93EF93FF938091B900887F06
:102F2000803609F49CC068F5883209F45BC090F4DF
:102F3000803109F454C038F4882309F4F6C088308D
:102F400009F44DC0F6C0883109F44CC0803209F450
:102F50005DC0EFC0803409F468C048F4803309F4E0
:102F600055C0883309F0E5C08093670AD8C0803522
:102F700009F44FC0883509F45DC0883409F0D9C020
:102F8000D6C0883909F4C7C0A8F4883709F467C0E7
:102F900038F4883609F463C0803709F460C0C9C0CA
:102FA000883809F4B8C0803909F45FC0803809F066
:102FB000C0C05BC0803B09F486C038F4803A09F495
:102FC00066C0883A09F47FC0B4C0803C09F4A7C049
:102FD000883C09F4A4C0883B09F48AC0AAC0809147
:102FE0008A0A10C09091890A8091880A981770F512
:102FF000E091890A81E08E0F8093890AF0E0E85918
:10300000F54F80818093BB0085EC86C08093670A72
:103010008EC0E091890A81E08E0F8093890A8091A9
:10302000BB00F0E0E859F54F80839091890A8091C8
:10303000880A6EC0E091890A81E08E0F8093890A28
:103040008091BB00F0E0E859F54F80838091CC0877
:1030500081116DC081E08093CB0884EA61C083E078
:103060008093CD081092B20ACFCF8091B20A8032FD
:1030700008F051C0E091B20A81E08E0F8093B20A4D
:103080008091BB00F0E0EE56F54F8083BDCF85EC1C
:103090008093BC001092CD088091B20A803230F447
:1030A000E091B20AF0E0EE56F54F10826091B20A5C
:1030B00070E0E091900AF091910A82E99AE0199506
:1030C0001092B20A36C084E08093CD0810928F0A25
:1030D0001092660AE0918D0AF0918E0A19958091FE
:1030E000660A811105C081E08093660A1092460A43
:1030F000E0918F0A81E08E0F80938F0AF0E0EA5B07
:10310000F54F80818093BB0090918F0A8091660A71
:10311000981708F479CF85E88093BC000AC085EC45
:103120008093BC001092CD0804C01092670A0E94E0
:10313000AC21FF91EF91BF91AF919F918F917F91C2
:103140006F915F914F913F912F910F900BBE0F9018
:103150000FBE0F901F901895DC015996ED91FC91D0
:103160005A973097B9F083899489A589B6894285A1
:10317000538564857585841B950BA60BB70B81154C
:1031800020E89207A105B10538F08FEF9FE7A0E096
:10319000B0E0089580E090E00895CF93DF931F9210
:1031A000CDB7DEB76983DC01ED91FC910280F3813C
:1031B000E02D41E050E0BE016F5F7F4F19950F9009
:1031C000DF91CF910895CF92DF92EF92FF920F930C
:1031D0001F93CF93DF9300D000D0CDB7DEB76C0143
:1031E000DC01ED91FC910284F385E02D2D833E837B
:1031F0004B835C8369837A831995D601ED91FC91A9
:103200000684F785E02D2D813E814B815C816981AB
:103210007A81C6011995D601ED91FC910688F7894E
:10322000E02DC60126960FB6F894DEBF0FBECDBFC7
:10323000DF91CF911F910F91FF90EF90DF90CF9092
:103240001994EF92FF920F931F93CF93DF9300D0C7
:1032500000D0CDB7DEB77C01DC01ED91FC9102849A
:10326000F385E02D2D833E834B835C8369837A83D2
:103270001995D701ED91FC910288F389E02D2D81FC
:103280003E814B815C8169817A81C7011995D701A3
:10329000ED91FC910688F789E02DC70126960FB6BF
:1032A000F894DEBF0FBECDBFDF91CF911F910F917C
:1032B000FF90EF901994EF92FF920F931F93CF938B
:1032C000DF9300D000D0CDB7DEB77C01DC01ED91FB
:1032D000FC910284F385E02D2D833E834B835C8338
:1032E00069837A831995D701ED91FC910088F18962
:1032F000E02D2D813E814B815C8169817A81C701FE
:103300001995D701ED91FC910688F789E02DC70149
:1033100026960FB6F894DEBF0FBECDBFDF91CF91DA
:103320001F910F91FF90EF901994EF92FF920F93DE
:103330001F93DC01ED91FC910684F785E02D780167
:1033400001E010E019951F910F91FF90EF90089503
:10335000EF92FF920F931F93DC01ED91FC91068495
:10336000F785E02D7801890121E030E019951F9162
:103370000F91FF90EF900895FC01818D928D009741
:1033800011F00C9479260895FC0183A9A6A5B7A590
:103390009C91892B8C9383A187FD0C948F2F08958A
:1033A000CF93DF93EC01898D9A8D009739F481E0FA
:1033B00090E09B838A8380E090E00BC0FC01138245
:1033C00012820E944A27E98DFA8D22813381232BB4
:1033D00071F7DF91CF910895AF92BF92CF92DF92B4
:1033E000EF92FF920F931F93CF93DF93EC0177FD42
:1033F00038C088859985681779079CF557FD31C0D5
:103400008A859B854817590764F569015A017B0134
:10341000E881F9810284F385E02DCE011995E881D8
:10342000F98102A4F3A5E02D01E010E021E030E0F5
:10343000A501B701CE011995B601CE010E94C606BD
:10344000E881F9810688F789E02DCE01DF91CF91DF
:103450001F910F91FF90EF90DF90CF90BF90AF90B2
:103460001994DF91CF911F910F91FF90EF90DF9012
:10347000CF90BF90AF900895EF92FF920F931F935C
:10348000CF93DF93EC0177FD22C08885998568177B
:103490007907ECF457FD1BC08A859B8548175907AF
:1034A000B4F47901E881F98102A4F3A5E02D01E0EB
:1034B00010E021E030E0CE011995B701CE01DF9197
:1034C000CF911F910F91FF90EF900C94C606DF9162
:1034D000CF911F910F91FF90EF9008950F931F933D
:1034E000CF93DF93EC018BA187FF1EC00C8D1D8D48
:1034F0002E8D3F8D90E040E052E16AE770E00417C6
:1035000015072607370740F4769567955795479531
:103510009F5F9630A1F797E081E09827892F806A16
:10352000869591700E94902F9BA9EEA5FFA58081A2
:10353000282F30E0892F90E0809590958223932367
:103540008083DF91CF911F910F910895CF93DF93E7
:10355000EC010E947926882311F01D8281E0DF9121
:10356000CF9108953F924F925F926F927F928F9288
:103570009F92AF92BF92CF92DF92EF92FF920F9302
:103580001F93CF93DF93CDB7DEB72C970FB6F89488
:10359000DEBF0FBECDBF5C01DC015B968D909C90C1
:1035A0005C971696CD90DD90ED90FC901997C11424
:1035B000D104E104F10439F0BFEFCB1ADB0AEB0AC6
:1035C000FB0A312C07C0F401C080D180E280F38077
:1035D00033243394F40181859285A385B4859C01BD
:1035E000AD012F5F3F4F4F4F5F4F29873A874B8782
:1035F0005C87260137011D821E821F821886F40116
:1036000081859285A385B4852D813E814F81588522
:10361000281739074A075B0708F063C089859A8530
:10362000AB85BC858C159D05AE05BF0550F482E0C9
:10363000C82ED12CE12CF12C92E0492E512C612C7A
:10364000712C9E012F5F3F4FB701A601C4010E945C
:103650008E25882309F445C089819A81AB81BC817C
:10366000892B8A2B8B2B41F0260137019FEF491ABA
:10367000590A690A790A05C0C414D504E604F70496
:1036800091F02D813E814F8158852F5F3F4F4F4FE5
:103690005F4F2D833E834F8358873FEFC31AD30A72
:1036A000E30AF30AACCF0FEF1FEF2FEF3FE0B301B8
:1036B000A201C4010E94EF24882399F0D501169637
:1036C0004D915D916D917C91199741155105610561
:1036D000710549F093018201C4010E94EF24811118
:1036E00002C080E02AC0D50116964D925D926D927F
:1036F0007C921997332051F0D301C2010196A11D8C
:10370000B11DF40180839183A283B383F50187897E
:10371000908DA18DB28D892B8A2B8B2B69F4D501CD
:1037200057964D925D926D927C925A9714968C9119
:103730001497806814968C9381E02C960FB6F894B9
:10374000DEBF0FBECDBFDF91CF911F910F91FF90D4
:10375000EF90DF90CF90BF90AF909F908F907F9031
:103760006F905F904F903F900895CF93DF93EC015F
:103770008091BC0A811109C081E08093BC0A8091CC
:103780006F09909170090E94902F60E08C81DF9109
:10379000CF910C943A1261E0FC0184810E943A12AC
:1037A0008091BC0A882321F01092BC0A0C948F2FC0
:1037B00008958EBD00000DB407FEFDCF8EB50895AF
:1037C0008FEFF7CF0F931F93CF93DF93EB012AD99E
:1037D0008B01F6DF8F3F41F025D9601B710B6C1711
:1037E0007D07B8F380E001C081E0DF91CF911F91A8
:1037F0000F910895CF93DF93EC018E81882379F0A8
:103800008F8198859C012F5F3F4F38872F838230AF
:10381000924010F4D5DFF4CFCE01BDDF1E82DF91E0
:10382000CF910895CF92DF92FF920F931F93CF9382
:10383000DF9300D01F92CDB7DEB76C01F62E29833F
:103840003A834B835C83D6DFC6018FDF6CE271E085
:10385000C601B8DF8F2D8064ACDF08E110E05C8129
:103860004B813A812981DA01C901002E04C0B69545
:10387000A795979587950A94D2F729833A834B8326
:103880005C8397DF0850110929813A814B815C8163
:10389000083F8FEF180739F7FF2029F0E8E0FE1204
:1038A00004C087E803C085E901C08FEF82DF10E024
:1038B00087DFF601828787FF04C01F3F11F01F5F7B
:1038C000F7CF0F900F900F900F90DF91CF911F9136
:1038D0000F91FF90DF90CF900895AF92BF92CF925B
:1038E000DF92EF92FF920F931F93CF93DF93EC0140
:1038F0006901C801820F931F8130924008F068C0AF
:103900008E81882371F088819981AA81BB814817B3
:1039100059076A077B0729F48F819885C816D9064D
:1039200088F5488359836A837B838B85833039F09C
:1039300089E0440F551F661F771F8A95D1F79A01BA
:10394000AB0161E1CE016EDF882319F083E08D8346
:103950003FC068D85B0134DF8A878F3F41F462D86B
:103960006A197B096D327140B0F38FE003C08E3F5E
:1039700029F08DE08D83CE010EDF2AC018861F82CC
:1039800081E08E838F8198858C159D0538F418DF32
:103990008F819885019698878F83F4CF6701E00E19
:1039A000F11ECE14DF0429F00BDFF60181936F01C5
:1039B000F8CF8F819885080F191F18870F83898585
:1039C000882319F00115124038F0CE0113DF04C02E
:1039D000CE01E1DE80E001C081E0DF91CF911F9157
:1039E0000F91FF90EF90DF90CF90BF90AF90089530
:1039F000EF92FF920F931F93CF93DF93EC01790126
:103A0000411551056105710511F482E134C08B85C2
:103A1000833039F089E0440F551F661F771F8A9560
:103A2000D1F79A01AB0168E1CE01FCDE882311F0E9
:103A300084E021C08EEFBDDE87018EEFF81AF80119
:103A400081918F01B6DE0E151F05C9F78FEFB1DE2C
:103A50008FEFAFDEB5DE8A878F71853029F081E187
:103A60008D83CE0198DE08C068E572E0CE01AADE43
:103A7000811106C085E18D83CE018DDE80E010C00E
:103A800020E030E0A9016DE0CE01CCDE811103C061
:103A900097DE882311F084E1EECFCE017CDE81E059
:103AA000DF91CF911F910F91FF90EF900895EF92CA
:103AB000FF920F931F93CF93DF93EC017B018A0159
:103AC0001B821A8288EE93E0A0E0B0E08C839D8395
:103AD000AE83BF8382EA92E0998388838DE190E090
:103AE0000E94C53B9A8F898F009779F02DE1F701ED
:103AF000DC0101900D922A95E1F74CE050E0B8010D
:103B0000CE010C960E94003E188EDF91CF911F913E
:103B10000F91FF90EF900895CF93DF931F92CDB751
:103B2000DEB741E050E0BE016F5F7F4F0E94E528A5
:103B3000019719F4898190E002C08FEF9FEF0F90F9
:103B4000DF91CF910895FC01818D928D009709F04E
:103B5000E3CF8FEF9FEF08950F931F93CF93DF93E2
:103B6000FC01818D928D0097B1F0EF01D5DF8C01C2
:103B70000F3F8FEF180791F0898D9A8DFC014285D8
:103B800053856485758541505109610971090E9409
:103B9000B526C80105C080E090E002C08FEF9FEF1E
:103BA000DF91CF911F910F910895CF93DF93FC0187
:103BB00083A187FF05C06EBD0DB407FEFDCF2EC0EB
:103BC00028E030E040E8A6A1B7A1842F862321F0A9
:103BD00080A99C91892B0AC090A98C91C82FD0E014
:103BE000892F90E0809590958C239D238C9392A9AA
:103BF000C2A5D3A58881A82FB0E0892F90E0809539
:103C000090958A239B23888382A9A2A5B3A59C9122
:103C1000892B8C93469521503109A9F6DF91CF91DC
:103C200008958F929F92AF92BF92CF92DF92EF92C0
:103C3000FF920F931F93CF93DF93EC01690158011B
:103C4000470128853985621773070CF05CC08A85A7
:103C50009B85481759070CF056C07B01EC0CFD1CE6
:103C6000D70111978A010A0D1B1DF8013197B7FD85
:103C70004AC0F7FD48C077FF03C0670160E070E00D
:103C800057FF03C0580140E050E0A217B3071CF0F3
:103C90006901C61AD70AE817F9071CF05C01A41AD3
:103CA000B50AE881F98102A4F3A5E02D850196010A
:103CB000CE0119959601D5010E94B93B6115710598
:103CC0008105910501F12BA127FD0AC06B017C0143
:103CD0000EC00DB407FEFDCF8EBC0DB407FEFDCFA8
:103CE000615071098109910970F09EBCF2CF692D74
:103CF000CE015BDF682DCE0158DF81E0C81AD10804
:103D0000E108F108A1F7DF91CF911F910F91FF908A
:103D1000EF90DF90CF90BF90AF909F908F900895DD
:103D2000CF93DF93EC019CA9ECA5FDA52081422F48
:103D300050E0292F30E0209530952423352320832F
:103D4000CE0133DF8CA9ECA5FDA59081892B808362
:103D5000DF91CF9108958F929F92AF92BF92CF92B1
:103D6000DF92EF92FF920F931F93CF93DF93EC01BB
:103D7000490181E0881A9108860E971EC401A0E0CF
:103D8000B0E04B01A12CB12C540199248824882A3D
:103D9000992AAA2ABB2A680181E0C81AD108C40E50
:103DA000D51EC601A0E0B0E06A01E12CF12C76013D
:103DB000DD24CC24C82AD92AEA2AFB2A6AE2CE01C9
:103DC000AFDF2BA16B2D77278827992727FF18C0F6
:103DD0006EBD0DB407FEFDCFC501AA27BB278EBD62
:103DE0000DB407FEFDCFBB27AB2D9A2D892D8EBDBF
:103DF0000DB407FEFDCF8EBC0DB407FEFDCF10C085
:103E0000CE01D3DEB50188279927CE01CEDE9927D2
:103E10008B2D7A2D692DCE01C8DE682DCE01C5DE31
:103E20006BE2CE017DDF2BA16F2D772788279927A5
:103E300027FF18C06EBD0DB407FEFDCFC701AA272E
:103E4000BB278EBD0DB407FEFDCFBB27AF2D9E2D2A
:103E50008D2D8EBD0DB407FEFDCFCEBC0DB407FE7B
:103E6000FDCF10C0CE01A1DEB70188279927CE0172
:103E70009CDE99278F2D7E2D6D2DCE0196DE6C2D2B
:103E8000CE0193DE6CE2CE01DF91CF911F910F91B5
:103E9000FF90EF90DF90CF90BF90AF909F908F906A
:103EA0003FCF0F931F93CF93DF931F92CDB7DEB712
:103EB0008C01DC01ED91FC910284F385E02D698396
:103EC00019956981611102C060E201C061E2C80117
:103ED00027DFD801ED91FC910688F789E02DC80114
:103EE0000F90DF91CF911F910F9119941F93CF9352
:103EF000DF93EC0163706D8B6230C1F0633001F1D0
:103F0000613051F080EF90E09987888780E491E0FC
:103F10009B878A8718E41DC080E491E09987888791
:103F200080EF90E09B878A8718E213C080EF90E0D3
:103F30009987888780E491E09B878A8718E809C081
:103F400080E491E09987888780EF90E09B878A875B
:103F500018EEE881F9810284F385E02DCE011995F0
:103F600066E3CE01DDDE612FCE011FDEE881F9813F
:103F70000688F789E02DCE01DF91CF911F9119942A
:103F8000BF92CF92DF92EF92FF920F931F93CF9346
:103F9000DF93EC01411551056105710521F440E005
:103FA00052E16AE770E04C8F5D8F6E8F7F8F88A142
:103FB00087FD07C061E00E949E1461E088A10E9415
:103FC0003A1261E089A10E949E1460E089A10E94DA
:103FD0003A128BA187FD16C061E08CA10E949E144D
:103FE00060E08CA10E943A1261E08BA10E949E14B5
:103FF00061E08BA10E943A128DA187FD03C060E0B1
:104000000E949E148BA187FD0E94932F8AA187FD99
:1040100021C061E00E949E1461E08AA10E943A12D0
:1040200064E670E080E090E00E94DA1460E08AA12B
:104030000E943A1264E670E080E090E00E94DA1498
:1040400061E08AA10E943A1268EC70E080E090E0A2
:104050000E94DA14E881F9810284F385E02DCE0113
:10406000199509EB13E07801EFEFEE1AFE0AF8015B
:104070006491662311F1CE0153DE0E5F1F4FF701ED
:10408000E490FE2DFF77BF2E6801FF2EFA948FEF8C
:10409000F81641F0F6016491CE0187DDFFEFCF1AEB
:1040A000DF0AF4CF0B0D111DE7FEDDCF68E770E0EE
:1040B00080E090E00E94DA14D6CFE881F98106888A
:1040C000F789E02DCE01199580EF90E099878887D8
:1040D00080E491E09B878A87DF91CF911F910F91B8
:1040E000FF90EF90DF90CF90BF9008950F931F93B4
:1040F000CF93DF931F92CDB7DEB78C01DC01ED913A
:10410000FC910284F385E02D69831995698166230A
:1041100019F0F80165A903C0D801D6966C91C801C1
:10412000FFDDD801ED91FC910688F789E02DC801EB
:104130000F90DF91CF911F910F9119944091660AD2
:10414000262F30E0240F311D21323105DCF420917F
:10415000CD082430C9F4FC0180E090E0861758F4C3
:104160003091660A2191DC01AA5BB54FA30FB11D06
:104170002C930196F3CF8091660A680F6093660ACC
:1041800080E0089581E0089582E008950895E09127
:10419000D1088091D008E81730F4F0E0ED51F54FE8
:1041A000808190E008958FEF9FEF08959091D1085E
:1041B0008091D008981750F4E92FF0E0ED51F54FB9
:1041C000208130E09F5F9093D10802C02FEF3FEF36
:1041D000C90108958091D00890E02091D108821BF8
:1041E00091090895CF92DF92EF92FF920F931F9360
:1041F000CF93DF937C01262F972F8A018091E20ACB
:10420000882391F0C62FD72F6E01C40ED51ECC1572
:10421000DD0569F06991D701ED91FC910190F08184
:10422000E02DC7011995F3CF642F822F87DFC801D6
:10423000DF91CF911F910F91FF90EF90DF90CF9082
:104240000895CF93DF931F92CDB7DEB76983209196
:10425000E20A2223D1F02091CE08203240F021E062
:1042600030E0FC013383228380E090E014C0809131
:10427000CF08E82FF0E0EE53F54F998190838F5FE0
:104280008093CF088093CE0804C061E0CE010196F0
:1042900055DF81E090E00F90DF91CF91089520915C
:1042A000CE089091C10A213208F04AC08091CD0811
:1042B0008111FCCF32E03093CD0831E03093CC084F
:1042C0003FEF3093670A1092890A2093880AA2EC84
:1042D000BAE048E65AE0FA013E2F341B321718F4D0
:1042E0003D913193F9CF10928A0A20918A0A990F51
:1042F000922B90938A0A9091CB08913061F410929E
:10430000CB0890918A0A9093BB009091BC0093FDDA
:10431000F8CF95EC01C095EE9093BC009091CD083C
:104320009230E1F39091670A9F3F79F08091670A9C
:10433000803241F08091670A803331F084E005C01B
:1043400081E003C082E001C083E01092CF081092A8
:10435000CE081092E20A089585ED8093BC0080910A
:10436000BC0084FDFCCF1092CD080895CF92DF925F
:10437000EF92FF920F93CF93DF931F92CDB7DEB7EB
:104380006C017901DC0114968C91149791E0909363
:10439000E20A8093C10A1092CF081092CE081596B7
:1043A0008D919C911697DC01ED91FC910190F0812B
:1043B000E02D49831995F60185819681DC01ED9107
:1043C000FC910190F081E02D4981642F1995F6014F
:1043D00085819681DC01ED91FC91402F50E00280B7
:1043E000F381E02DB7011995F60187818F3F71F4B4
:1043F000D60115968D919C9116970F90DF91CF91D4
:104400000F91FF90EF90DF90CF9049CFF601878119
:104410000E941212892BD1F3EBCFCF92DF92EF9251
:10442000FF920F93CF93DF93CDB7DEB7A0970FB670
:10443000F894DEBF0FBECDBF6C01862FFB010E2F9F
:10444000081B9191E02EF12C992341F0A1E0B0E0FE
:10445000AC0FBD1FAE0DBF1D9C93F1CF9E012F5F12
:104460003F4F45E062E0C60181DFC701A0960FB66D
:10447000F894DEBF0FBECDBFDF91CF910F91FF90BB
:10448000EF90DF90CF9008950F93CF93DF931F921B
:10449000CDB7DEB7698301E09E012F5F3F4F45E056
:1044A00062E064DF61E070E080E090E00E94DA1496
:1044B00081E090E00F90DF91CF910F9108950F93DD
:1044C000CF93DF9300D0CDB7DEB76450643088F46B
:1044D000E62FF0E0EC54FD4F208127FD0AC0298330
:1044E0005A834B8303E09E012F5F3F4F42E068E019
:1044F0003DDF0F900F900F90DF91CF910F910895B6
:10450000EF92FF920F931F93CF93DF9300D0CDB71D
:10451000DEB76450643008F5E62FF0E0E055FD4F5B
:10452000108117FD1AC0622F9A017C01603151F091
:10453000AFEFBFEF0E94C13A2FEF30E040E050E014
:104540000E94793A19833A832B8303E09E012F5FFF
:104550003F4F41E068E0C70109DF0F900F900F90D7
:10456000DF91CF911F910F91FF90EF9008952F92BF
:104570003F924F925F926F927F928F929F92AF92F3
:10458000BF92CF92DF92EF92FF920F931F93CF9340
:10459000DF9300D000D0CDB7DEB79E838D83562E3B
:1045A000442E3C832B834701C701880F991F880F36
:1045B000991F3C0125E0621A710810E0FF24F39472
:1045C000202E312C35ECE32E101708F0CDC0AD8134
:1045D000BE8114968C911497F092E20A8093C10ADE
:1045E0001092CF081092CE0815968D919C91169737
:1045F000DC01ED91FC910190F081E02D652D199584
:10460000ED81FE8185819681DC01ED91FC91019027
:10461000F081E02D642D1995ED81FE8187818F3F1A
:1046200079F4AD81BE8115968D919C91169737DEF8
:10463000B2E08B16910460F0C3010197F1F708C056
:10464000ED81FE8187810E941212892BC9F3E9CF87
:10465000AD81BE8117968C918F3F21F4ED81FE8153
:10466000348109C0AD81BE8117968C910E941212CF
:10467000892BC1F3F3CF8091CD088111FCCFC1010B
:10468000811B91098132910514F080E290E0282F7E
:10469000813208F020E2F092CD08F092CC08BFEF12
:1046A000B093670A1092890A4FEF420F4093880A2D
:1046B000F0928A0A40918A0A330F342B30938A0A87
:1046C0003091CB08313069F41092CB0830918A0ACE
:1046D0003093BB003091BC0033FDF8CFE092BC00BA
:1046E00003C0E5EEE093BC003091CD083130E1F33A
:1046F0003091890A321710F42091890AA8E6BAE0AD
:10470000E3EEFAE03E2F43EE5AE0341B321718F482
:104710003D913193F7CF1092D1082093D008A12C6E
:10472000B12C6C01DD24812F8A0DAC14BD04D4F4AE
:104730002B813C81280F311D3A832983AD81BE81B5
:1047400015968D919C911697DC01ED91FC91028458
:10475000F385E02D1995E981FA818083FFEFAF1A87
:10476000BF0AE1CF182F30CF26960FB6F894DEBFE0
:104770000FBECDBFDF91CF911F910F91FF90EF90B2
:10478000DF90CF90BF90AF909F908F907F906F9071
:104790005F904F903F902F900895EF92FF920F936C
:1047A0001F93CF93DF931F921F92CDB7DEB7633075
:1047B00059F020F4623021F540E009C0643031F056
:1047C0006530F1F443E003C041E001C042E0495FDD
:1047D00024EFE22EFF24F39402E09E012F5F3F4F6F
:1047E00069E0C5DE098110E0102F00278A81082BBF
:1047F00061E070E080E090E00E94DA14C80102C03D
:1048000080E090E00F900F90DF91CF911F910F917A
:10481000FF90EF900895EF92FF920F93CF93DF9365
:1048200000D01F92CDB7DEB728EEE22E23E0F22EA5
:1048300004E09E012F5F3F4F44E060E098DE298155
:104840006A81862F90E0A0E0B0E0DC0199278827FC
:10485000B22B2C81822B2B81BC01CD01722B0E94AB
:10486000663920E030E040E857E30E94C5390F90F8
:104870000F900F900F90DF91CF910F91FF90EF90DD
:104880000895EF92FF920F93CF93DF9300D01F9282
:10489000CDB7DEB72DE7E22EF12C04E09E012F5FAD
:1048A0003F4F42E060E063DE29816A81862F90E01D
:1048B000A0E0B0E0DC0199278827B22B2C81822B65
:1048C0002B81BC01CD01722B0F900F900F900F9098
:1048D000DF91CF910F91FF90EF9008958091CA06DC
:1048E000882399F1409100025091010260910202E7
:1048F000709103022BEC36E08091C8069091C906B6
:1049000077D8811102C080E008954091BD0A50918E
:10491000BE0A6091BF0A7091C00A41155105610538
:10492000710589F02BEC36E08091C8069091C9069C
:104930005FD8882341F31092BD0A1092BE0A1092EC
:10494000BF0A1092C00A1092CA0681E008958F92A1
:104950009F92AF92BF92EF92FF920F931F93CF93CC
:104960004B015C01C42F8091000290910102A09143
:104970000202B091030288159905AA05BB05F9F05A
:10498000ADDF811102C080E020C08BECE82E86E014
:10499000F82E00E012E020E030E0B501A4018091A3
:1049A000C8069091C9060E946D1C882361F380920D
:1049B000000290920102A0920202B0920302809142
:1049C000CA06C82BC093CA0681E0CF911F910F91F0
:1049D000FF90EF90BF90AF909F908F9008954F926F
:1049E0005F926F927F928F929F92AF92BF92CF927F
:1049F000DF92EF92FF920F931F93CF93DF93EC011F
:104A00006A017B01280139014230510561057105B8
:104A100010F480E072C089859A85AB85BC850196CB
:104A2000A11DB11D84179507A607B70790F38B88C2
:104A30009C88AD88BE888F89803129F4BB27AF2D33
:104A40009E2D8D2D09C0DB01CA0147E0B695A795C3
:104A5000979587954A95D1F7880E991EAA1EBB1E79
:104A60008091000290910102A0910202B091030294
:104A700088169906AA06BB0679F48F89803199F4C5
:104A8000DD24EE24FF24C601880F991FFC01E553A5
:104A9000F94F5182408218C040E0C501B40157DF90
:104AA0008111EBCFB6CFE894C7F8DD24EE24FF24C4
:104AB000C601880F991F880F991FFC01E553F94F14
:104AC00040825182628273828091CA0681608093A3
:104AD000CA068A89823080F08D819E81AF81B88537
:104AE000880E991EAA1EBB1E8092BD0A9092BE0A15
:104AF000A092BF0AB092C00A81E0DF91CF911F91CE
:104B00000F91FF90EF90DF90CF90BF90AF909F906C
:104B10008F907F906F905F904F9008958F929F92AB
:104B2000AF92BF92CF92DF92EF92FF920F931F93BB
:104B3000CF93DF93FC0181859285A385B48501968F
:104B4000A11DB11D84179507A607B70710F480E0D3
:104B50005BC083899489A589B689C789C03129F446
:104B6000852E962EA72EBB2409C04A015B01C7E003
:104B7000B694A79497948794CA95D1F7E9016A01EE
:104B80007B018F01BC01CD01680D791D8A1D9B1D24
:104B90008090000290900102A0900202B090030267
:104BA000681579058A059B0599F4F8018789803194
:104BB000A1F4B701A601552766277727440F551F93
:104BC000FA01E553F94F80819181A0E0B0E017C070
:104BD00040E0BDDE8111E9CFBACFB701A6014F7722
:104BE000552766277727440F551F440F551FFA0195
:104BF000E553F94F80819181A281B381BF70888391
:104C00009983AA83BB8381E0DF91CF911F910F919C
:104C1000FF90EF90DF90CF90BF90AF909F908F90DC
:104C200008954F925F926F927F92AF92BF92CF9210
:104C3000DF92EF92FF920F931F93CF93DF9300D0F9
:104C40001F92CDB7DEB78C0149835A836B837C8377
:104C50005901C12CD12C7601412C82E0582E612CB7
:104C6000712C49815A816B817C819E012F5F3F4F5E
:104C7000C80154DF882351F1D301C201F801058432
:104C800004C0880F991FAA1FBB1F0A94D2F7C80E31
:104C9000D91EEA1EFB1E49815A816B817C8187895E
:104CA000803129F088EF9FEFAFEFBFE004C088EFBD
:104CB0009FEFA0E0B0E0481759076A077B0788F22A
:104CC000F501C082D182E282F38281E00F900F90E1
:104CD0000F900F90DF91CF911F910F91FF90EF9068
:104CE000DF90CF90BF90AF907F906F905F904F908C
:104CF0000895CF93DF93EC018D81882391F18C810E
:104D000087FF2CC06E857F858889998941E01FDEE9
:104D1000882339F1EA8980E2E89FF0011124DF015C
:104D2000A553B94F1097E9F08D81823050F44B892B
:104D30005C896D897E895C964D935D936D937C93C0
:104D40005F978F89988DA98DBA8DE553F94F938F11
:104D5000828FB58BA48B8C818F778C83DF91CF91E1
:104D6000BDCD80E0DF91CF9108958F929F92AF9259
:104D7000BF92CF92DF92EF92FF920F931F93CF9348
:104D8000DF93EC018D81811102C080E076C00B8938
:104D90001C892D893E890417150726073707A8F3B4
:104DA0006A017B01823029F4CA86DB86EC86FD86A7
:104DB0000DC0C114D104E104F10451F41E821F821C
:104DC000188619861A861B861C861D8681E055C0AA
:104DD0008A849B84AC84BD84EB8DFC8D258530E07A
:104DE000275F3F4FB501A401415051096109710985
:104DF000022E04C076956795579547950A94D2F789
:104E0000D701C6010197A109B10904C0B695A795BC
:104E1000979587952A95D2F784179507A607B70720
:104E200020F089288A288B2849F44F89588D698D6C
:104E30007A8D4E835F836887798704C0841B950BC6
:104E4000A60BB70B4C015D018E010A5F1F4F811449
:104E50009104A104B10409F4A7CF4E815F81688554
:104E6000798598018B8D9C8D59DE91E0891A910886
:104E7000A108B1088111EBCF88CFDF91CF911F91AD
:104E80000F91FF90EF90DF90CF90BF90AF909F90E9
:104E90008F9008952F923F924F925F926F927F92E0
:104EA0008F929F92AF92BF92CF92DF92EF92FF923A
:104EB0000F931F93CF93DF9300D01F92CDB7DEB730
:104EC0008C015B011A01DC0115968C9115978130DC
:104ED000C1F414968C9181FF14C082FF1AC0F801AE
:104EE000438954896589768982859385A485B585AA
:104EF00084179507A607B70761F0C80136DF81114F
:104F000008C081E090E0F8019383828380E090E024
:104F100035C1610183C0D8015B968D919C915C97EE
:104F2000FC01248121502A013B0139E076946794E9
:104F3000579447943A95D1F7722E74207A01F1E094
:104F4000FF22772009F476C080E092E08E199F0955
:104F500046018C159D0508F44C01D8015B962D91F6
:104F60003C915C9716968D919D910D90BC91A02DD2
:104F70000297A109B109F901058404C0880F991F9E
:104F8000AA1FBB1F0A94D2F746855785608971898D
:104F9000840F951FA61FB71F9C01AD01270D311D62
:104FA000411D511D29013A01811432E0930609F097
:104FB00087C08091000290910102A0910202B091FD
:104FC000030284159505A605B70559F48FEF9FEFE9
:104FD000DC018093000290930102A0930202B0933F
:104FE00003029501B301A2018091C8069091C90600
:104FF0000E94F81C882309F484CF9EEFB91AC818C0
:10500000D908F80182859385A485B585880D991DF9
:10501000A11DB11D82879387A487B587D8011A96F1
:105020004D915D916D917C911D97C114D10409F052
:1050300072CF84C0E114F10409F086CF16964D9129
:105040005D916D917C91199741155105610571052F
:1050500059F457968D919D910D90BC91A02D00977C
:10506000A105B10539F520C09E012F5F3F4F56DDE8
:10507000882309F44CCF89819A81AB81BC81F801E6
:10508000238D348DF9012789203129F048EF5FEF16
:105090006FEF7FE004C048EF5FEF60E070E08417DF
:1050A0009507A607B70730F0C8010E94B21A811110
:1050B0004BCF27CFF80186839783A087B18744CF52
:1050C000E114F10421F5D8011A964D915D916D918D
:1050D0007C911D9753968D919D910D90BC91A02D23
:1050E000481759076A077B0790F0F8DB882309F413
:1050F00008CF409200025092010260920202709228
:1051000003028091CA0681608093CA0607C041E00D
:10511000C301B2011CDC882309F4F3CED501F701E9
:10512000E553F94FCF01880D991DE817F90719F0DC
:105130002D912193FACFA80CB91C61CF53968D9174
:105140009D910D90BC91A02D84179507A607B707D8
:1051500040F4F801438B548B658B768B8481806897
:105160008483D80114968C9183FD02C0C10106C0CE
:10517000C801BFDD882309F4C4CEF8CF0F900F908B
:105180000F900F90DF91CF911F910F91FF90EF90B3
:10519000DF90CF90BF90AF909F908F907F906F9057
:1051A0005F904F903F902F900895CF93DF931F9281
:1051B000CDB7DEB7698341E050E0BE016F5F7F4F3E
:1051C00069DE0F90DF91CF9108952F923F924F9219
:1051D0005F926F927F928F929F92AF92BF92CF9287
:1051E000DF92EF92FF920F931F93CF93DF93EC0127
:1051F0006B014A018D81811103C08FEF9FEFD5C0F4
:105200008C8180FFFACF4B885C886D887E884A85C8
:105210005B856C857D85C401A0E0B0E093018201CF
:10522000041B150B260B370B081719072A073B071A
:1052300018F44201841A950A54011E0126E0220E38
:10524000311CA114B10409F47DC04A855B856C85CD
:105250007D852A0181E05822ED818A019B0189E048
:1052600036952795179507958A95D1F78B8D9C8D47
:10527000E23061F4FC01828D938DA48DB58DBC016B
:10528000CD01600F711F821F931F3EC0FC0174800F
:105290007A94702241145104C1F4711016C0452B48
:1052A000462B472B49F48F89988DA98DBA8D8E8313
:1052B0009F83A887B98709C04E815F8168857985FA
:1052C00091012CDC882309F498CFEB8DFC8D8E8125
:1052D0009F81A885B9850297A109B109058404C0F9
:1052E000880F991FAA1FBB1F0A94D2F746855785BE
:1052F00060897189840F951FA61FB71FBC01CD015E
:10530000670D711D811D911D20E032E024193509C2
:1053100035012A153B0508F439012C8126FD04C00E
:105320006114F2E07F0681F4009100021091010205
:1053300020910202309103026017710782079307E0
:10534000A9F402C0C40131C040E001DB882309F4A4
:1053500054CFF201E553F94FD601CF01860D971DC9
:10536000E817F90789F021912D93FACF760183018F
:105370009201AB01BC018091C8069091C9060E94C0
:105380006D1C882309F439CFC60CD71C8A859B85F0
:10539000AC85BD85860D971DA11DB11D8A879B8794
:1053A000AC87BD87A618B7084CCFDF91CF911F916E
:1053B0000F91FF90EF90DF90CF90BF90AF909F90B4
:1053C0008F907F906F905F904F903F902F900895B7
:1053D0000895FC016370658B8481958126813781F6
:1053E000613039F0633029F09187808733872287D5
:1053F0000895318720879387828708952F923F925F
:105400004F925F926F927F928F929F92AF92BF92D4
:10541000CF92DF92EF92FF920F931F93CF93DF9380
:10542000CDB7DEB76C970FB6F894DEBF0FBECDBF19
:105430009C8F8B8F5B011A011F830E833701C982FA
:10544000DC0158964D915C9159974115510509F031
:10545000E5C018968D919C911997681779070CF003
:10546000CAC11A968D919C911B97281639060CF08B
:10547000C2C18C2C912CFB0136E0C39EE00DF11DC6
:105480001124FB87EA871E161F060CF0B4C1C40165
:1054900033E0880F991F3A95E1F79D878C87820D3D
:1054A000931D181619060CF0A6C157968C91811100
:1054B00003C0203B08F02F5FAB8DBC8DED91FC91BC
:1054C00011970284F385E02DCD012A8F19952A8D3D
:1054D000B5E02B9F90011124F5013596FF87EE87EB
:1054E000BB82AA822501A9014A195B09598B488B05
:1054F000C10108969B8B8A8BE889F989E40DF51D1B
:10550000E85DFB4F9491988761013D822C82A885CC
:10551000A0FF13C0AB8DBC8DED91FC91B981B13072
:1055200031F40484F585E02D2E813F8116C0068478
:10553000F785E02DEE80FF801AC0EE81FF816E16A8
:105540007F06F1F0AB8DBC8DED91FC91B981B1304E
:1055500051F40484F585E02D9301A601B2018B8DF1
:105560009C8D19950DC00684F785E02D730184018B
:1055700094014C815D816A817B818B8D9C8D199515
:10558000E885E695E887FFEFCF1ADF0A2C813D8199
:10559000280D391D3D832C834A895B89C416D506A5
:1055A00009F0B5CF5FEF451A550A8A819B81880DB6
:1055B000991D9B838A83AE85BF854A165B0609F0D9
:1055C0009BCFEE81FF816E167F0609F4F2C0EB8D52
:1055D000FC8DA081B181F981F13079F4B5016B5F67
:1055E0007F4F5096ED91FC915197830128E030E078
:1055F000A1018B8D9C8D1995DCC06A857B8568190E
:1056000079091E96ED91FC911F9773010C851D85FC
:105610009401A1018B8D9C8D1995CBC0FA01349614
:105620009491329765917491291BCB01B7E02B9F20
:10563000800D911D1124FA01259134913B8B2A8B09
:10564000FC01459154915B834A83FC013296C490DE
:10565000319654915E87329614913196D490898117
:10566000823058F0612E012E000C7708AD2D0D2CE4
:10567000000CBB0BB987A88704C019861886612C5B
:10568000712CAB8DBC8DED91FC9111970284F3854B
:10569000E02DCD011995B9818B2E912C689CC0010C
:1056A000699C900D789C900D1124FC01EA0DFB1D66
:1056B000FD87EC871C82712C612CE12F110FFF0BF1
:1056C00095012E0F3F1F3B872A87AC0CB11CA5010B
:1056D0004E0F5F1F5F8B4E8BC1018D0D911DD7FC4F
:1056E0009A95998F888F4E85641608F062C0862D32
:1056F00090E048855985480F591F489D9001499D64
:10570000300D589D300D1124D901A20DB31DB98B58
:10571000A88BAA84BB844C845D84DC80BA85DB1AA8
:10572000E88DF98DE80FF91FFD8BEC8B8D2D8A0D1F
:105730002E893F89A216B306B9F1877061F48A8178
:105740009B810196EA89FB89AA81BB81EA0FFB1F35
:1057500074909B838A8377FE20C0AB8DBC8DED91C6
:10576000FC91B981B13061F40484F585E02D2E817E
:105770003F814C895D89B5018B8D9C8D19950DC03C
:105780000684F785E02DEE80FF808401940148892E
:105790005989B2018B8D9C8D1995770CEFEFAE1A5C
:1057A000BE0A480C591CC2CF3C813C0D3C8363941B
:1057B0009ACFAB8DBC8DED91FC9111970688F7893E
:1057C000E02DCD016C960FB6F894DEBF0FBECDBFB5
:1057D000DF91CF911F910F91FF90EF90DF90CF90CD
:1057E000BF90AF909F908F907F906F905F904F9001
:1057F0003F902F9019946C960FB6F894DEBF0FBEB1
:10580000CDBFDF91CF911F910F91FF90EF90DF906F
:10581000CF90BF90AF909F908F907F906F905F9050
:105820004F903F902F900895AF92BF92CF92EF92FA
:10583000FF920F931F93CF93DF93EC01262F888D58
:10584000998D009709F03FC06A3059F41D861C8677
:105850002C898E859F8538E0239F800D911D112412
:1058600040C06D3009F4A8C08E898823C1F03C89FE
:105870008C859D8546E0349F800D911D11244885BF
:105880005985481759075CF41D861C868E859F85AF
:1058900048E0349F800D911D11249F878E87EA88F0
:1058A000FB88088919894E855F856C857D85CC8844
:1058B000CE01A4DD2C898C859D8536E0239F800D4B
:1058C000911D112442C06A3079F41D861C862C89F2
:1058D000FC013696E4918E859F852E9F800D911D4B
:1058E00011249F878E8768C06D3009F465C0FC0164
:1058F00034963491631708F45FC03196E491E6174B
:1059000008F45AC0FC013296A590B490462F50E09E
:10591000431B510937E0349FB001359F700D1124AE
:10592000A60EB71EF501329634913196E4913323D9
:1059300011F0E1110DC0F5013496E4912C898C85AC
:105940009D85E29F800D911D11249D878C8734C019
:10595000F501359644915E89552311F16C89E32F49
:10596000F0E0E40FF11D47FDFA956E9FD0016F9FA7
:10597000B00D11244C855D854A0F5B1FE885F985C4
:10598000E417F5076CF41D861C86FC013696E4913D
:105990008E859F856E9F800D911D11249F878E8718
:1059A000EA88FB88088919894E855F856C857D8525
:1059B000CC88CE0123DDBFCF81E090E0DF91CF9195
:1059C0001F910F91FF90EF90CF90BF90AF900895EF
:1059D0006F927F928F929F92AF92BF92CF92DF92FF
:1059E000EF92FF920F931F93CF93DF93EC014B0144
:1059F0005A0169013801E881F9810284F385E02DBB
:105A00001995E881F9810288F389E02D87019601D3
:105A1000A501B401CE011995E881F981A501460DD2
:105A2000571D415051090288F389E02D9601B401B8
:105A3000CE011995E881F9810088F189E02D930163
:105A4000A501B401CE011995E881F981C80CD91CD2
:105A5000B601615071090088F189E02D9301A5011B
:105A6000CE011995E881F9810688F789E02DCE01EC
:105A7000DF91CF911F910F91FF90EF90DF90CF902A
:105A8000BF90AF909F908F907F906F901994CF921E
:105A9000DF92EF92FF920F931F93CF93DF9300D08B
:105AA00000D0CDB7DEB76C01DC01ED91FC9162173F
:105AB000730789F4041715072CF4942F852FA80178
:105AC000092F182F041B150B98012F5F3F4F048CD3
:105AD000F58DE02D12C04017510709F5261737073D
:105AE0002CF4962F872FB901292F382F261B370B1F
:105AF0002F5F3F4F068CF78DE02D8701C60119956A
:105B000026960FB6F894DEBF0FBECDBFDF91CF91C2
:105B10001F910F91FF90EF90DF90CF900895028436
:105B2000F385E02D2D833E834B835C8369837A83E9
:105B30001995D601ED91FC910488F589E02D2D8110
:105B40003E814B815C8169817A81C6011995D601BC
:105B5000ED91FC910688F789E02DC60126960FB6D7
:105B6000F894DEBF0FBECDBFDF91CF911F910F9193
:105B7000FF90EF90DF90CF901994EF92FF920F93E8
:105B80001F93DC01ED91FC9111971A960D911C91D8
:105B90001B9718962D913C91199700A0F1A1E02D2B
:105BA0007B0140E050E060E070E019951F910F919B
:105BB000FF90EF9008954F925F926F927F928F9235
:105BC0009F92AF92BF92CF92DF92EF92FF920F938C
:105BD0001F93CF93DF931F921F92CDB7DEB76C0157
:105BE0005A0139014801DC01ED91FC910284F385F1
:105BF000E02D69837A8319956981462E7A81572E23
:105C0000640C751CD601ED91FC91461457046CF49C
:105C10000088F189E02D87019401A501B201C60138
:105C20001995BFEF4B1A5B0AEDCF0688F789E02D77
:105C3000C6010F900F90DF91CF911F910F91FF90B0
:105C4000EF90DF90CF90BF90AF909F908F907F901C
:105C50006F905F904F901994AF92BF92CF92DF9266
:105C6000EF92FF920F931F93CF93DF9300D01F9279
:105C7000CDB7DEB75C016901DC01ED91FC910284D6
:105C8000F385E02D4B835C8369837A831995D50175
:105C9000ED91FC9169817A819B012C0D3D1D215074
:105CA00031090488F589E02D78014B815C818A01F6
:105CB000C5011995D501ED91FC910688F789E02D74
:105CC000C5010F900F900F900F90DF91CF911F9112
:105CD0000F91FF90EF90DF90CF90BF90AF9019940D
:105CE000AF92BF92CF92DF92EF92FF920F931F93EA
:105CF000CF93DF9300D01F92CDB7DEB75C0169016F
:105D0000DC01ED91FC910284F385E02D4B835C83F3
:105D100069837A831995D501ED91FC914B815C8162
:105D2000C40ED51EB1E0CB1AD1080488F589E02D48
:105D30007801860169817A819B01C5011995D50198
:105D4000ED91FC910688F789E02DC5010F900F9029
:105D50000F900F90DF91CF911F910F91FF90EF90D7
:105D6000DF90CF90BF90AF9019940895EF92FF927B
:105D70000F931F93DC01ED91FC9100A0F1A1E02DA8
:105D800019951F910F91FF90EF9008950F931F9316
:105D9000DC01ED91FC91068CF78DE02D19951F919A
:105DA0000F9108950F931F93DC01ED91FC91048CEA
:105DB000F58DE02D19951F910F910895DC01ED915E
:105DC000FC910084F185E02D199408952F923F9263
:105DD0004F925F926F927F928F929F92AF92BF92FB
:105DE000CF92DF92EF92FF920F931F93CF93DF93A7
:105DF00000D0CDB7DEB74C017B836A836A015901BD
:105E000017019801241B350B37FF03C031952195ED
:105E10003109C5014A815B81841B950B97FF03C043
:105E200091958195910951E059838217930714F058
:105E300019820BC09A2D8B2D5801092F182F9A818A
:105E40008B81DB82CA82C92ED82E8A819B81A816BB
:105E5000B9065CF49C2D8D2D6801092F182F9A81AD
:105E60008B81BB82AA82A92EB82E2501AA81BB8173
:105E70004A1A5B0A38016C187D0877FE03C07194DA
:105E800061947108720157FE03C0BFEFEB1AFB0A61
:105E9000F594E794C016D1061CF00FEF1FEF1FC05A
:105EA00001E010E01CC0D401ED91FC91B9810484A3
:105EB000F585E02D9101BB23C1F04A815B81B601DC
:105EC000C4011995E618F708F7FE04C0C00ED11EEC
:105ED000E40CF51CEA81FB813196FB83EA834A815D
:105EE0005B81A416B506FCF604C0A6016A817B811D
:105EF000E7CF0F900F900F90DF91CF911F910F91EF
:105F0000FF90EF90DF90CF90BF90AF909F908F90D9
:105F10007F906F905F904F903F902F9008950895DD
:105F20008CBD9DBD0895CF93CFB7F8948091030B9E
:105F3000811127C0EEE8F3E08491EEE2F3E0949162
:105F4000E82FF0E0EE0FFF1FE156FC4FA591B49152
:105F5000EC91E92321F461E085E30E943A1261E0CB
:105F600085E30E949E148CB580618CBD8CB58064E5
:105F70008CBD61E084E30E949E1461E083E30E9493
:105F80009E148091030B8F5F8093030BCFBFCF9143
:105F900008953F924F925F926F927F928F929F925D
:105FA000AF92BF92CF92DF92EF92FF920F931F9327
:105FB000CF93DF9300D000D0CDB7DEB77C016B016B
:105FC0003A0100E010E0512C412CA12CB12C4801E9
:105FD000F601848195810817190738F50F5F1F4F67
:105FE0009801A401B601CE0101960E94B41668EC96
:105FF00075E0CE0101960E946815382ECE010196FB
:106000000E948216332019F3C5010196A614B70425
:1060100041F49401452D542DB601C7010E94B416D8
:1060200009C0502E412E5C01D2CF62E975E0C70154
:106030000E94A016C70126960FB6F894DEBF0FBEC9
:10604000CDBFDF91CF911F910F91FF90EF90DF9027
:10605000CF90BF90AF909F908F907F906F905F9008
:106060004F903F9008956F927F928F929F92AF9240
:10607000BF92CF92DF92EF92FF920F931F93CF9335
:10608000DF93CDB7DEB762970FB6F894DEBF0FBED1
:10609000CDBF8C0162E975E08CEC99E00E94681537
:1060A0008111C5C16091CC097091CD09611571054F
:1060B00049F04091D0095091D10986EC99E00E94B5
:1060C000631604C086EC99E00E945116F801A48082
:1060D000B580F6E3AF16B10460F4B801CE010196C5
:1060E0000E948716CE0101960E94B80E0E94B00E43
:1060F0007DC0C50165E370E00E949D3BA81AB90A06
:1061000095E3C92ED12CE12CF12CEA14FB040CF000
:106110004AC0A701772473944A018FEF881A980A1E
:106120009401B801CE0101960E94B41668EC75E0A6
:10613000CE0101960E946815682ECE0101960E943C
:1061400082166110712CA4018C149D0429F796010C
:10615000A701B801CE0101967720A1F00E94B416E4
:10616000BE016F5F7F4FCE0107960E948716CE015A
:1061700007960E94B80E0E94B00ECE0107960E94AC
:10618000821606C00E94B416CE0101960E94B00E7F
:10619000CE0101960E948216E5E3EE0EF11CF5E3B6
:1061A000CF0ED11CB2CFF80124813581C90165E33E
:1061B00070E00E949D3B0097E9F0A901481B590B34
:1061C000B801CE0101960E94B416BE016F5F7F4FE9
:1061D000CE0107960E948716CE0107960E94B80E40
:1061E0000E94B00ECE0107960E948216CE01019643
:1061F0000E9482166CEC79E0CE0107960E94871609
:10620000CB84DC8400E010E0E12CF12C0C151D05A2
:10621000F4F40F5F1F4FA801415051099801BE01CE
:10622000695F7F4FCE0101960E94B41668EC75E05D
:10623000CE0101960E946815B82ECE0101960E94EB
:106240008216BB2019F3FFEFEF1AFF0ADFCFCE0152
:1062500007960E9482168701015011098FE1E81606
:10626000F1040CF442C068EC75E0CE0101960E9486
:10627000A016C090D009D090D109C114D10479F1F1
:10628000E090CC09F090CD0969817A81C7010E9424
:106290000F3E009721F0BC016E197F0902C06FEF1D
:1062A0007FEF6F5F7F4FD9F0C616D70608F4B601AF
:1062B000A601461B570B5093D1094093D0096E0D90
:1062C0007F1DC7010E94003EE091CC09F091CD09ED
:1062D0008091D0099091D109E80FF91F1082CE0169
:1062E00001960E9482167801B6CF1092170A10927A
:1062F000160A83E0EE0CFF1C8A95E1F7F092190A6A
:10630000E092180A8FEF9FEF90931D0A80931C0A6A
:1063100090931B0A80931A0A81E080931E0A6801F9
:106320008FEFC816D80609F488C06CEC79E0CE016E
:1063300007960E948716A601BE01695F7F4FCE01B6
:10634000019627DECE0107960E9482168091180AD8
:106350009091190A08971092170A1092160A9093B2
:10636000190A8093180A66EC79E0CE0107960E941C
:106370008716A601BE01695F7F4FCE010D9609DE2B
:106380002D813E8189899A892817390719F58981D4
:106390009A816D857E85009719F061157105A9F4C4
:1063A0006115710551F02115310539F0FB0180812E
:1063B00090E09195819591090AC0009769F0232B8F
:1063C00059F0FC01808190E002C00E94F03D11E094
:1063D000892B19F010E001C011E0CE010D960E944A
:1063E0008216CE0107960E948216111118C04091A4
:1063F000180A5091190AE12CF12C08E010E020E471
:1064000031E060E070E08AE09AE00E94E3184D819C
:106410005E8169817A818AE09AE00E94EE12CE0163
:1064200001960E948216F1E0CF1AD10879CF60E080
:1064300070E08AE09AE0A1DB35CE62960FB6F89460
:10644000DEBF0FBECDBFDF91CF911F910F91FF90A7
:10645000EF90DF90CF90BF90AF909F908F907F9004
:106460006F90089540E050E062E975E08CEC99E0AF
:106470000C946316CF92DF92EF92FF920F931F93CB
:10648000CF93DF93CDB7DEB72C970FB6F894DEBF6E
:106490000FBECDBF6B017C018A016CE975E0CE01B6
:1064A00001960E94A016B701A601CE0101960E9496
:1064B000E41561EC75E0CE0101960E94431620E0E0
:1064C00030E040E151E4C701B6015FD720E030E0A1
:1064D00040EA50E40E94353B20E030E040E052E4E6
:1064E0000E94D13AAB01BC01CE0101960E94B415C5
:1064F00066EC75E0CE0101960E9443166AEC75E0E9
:10650000CE0101960E944316B801CE0101960E9469
:1065100014166CEE75E0CE0101960E944316BE0182
:106520006F5F7F4FCE0107960E948716CE010796B8
:106530009ADDCE0107960E948216CE0101960E9436
:1065400082162C960FB6F894DEBF0FBECDBFDF913A
:10655000CF911F910F91FF90EF90DF90CF90089512
:10656000CF92DF92EF92FF920F931F93CF93DF931F
:10657000CDB7DEB72C970FB6F894DEBF0FBECDBFF8
:106580006B017C018A016EEE75E0CE0101960E94DE
:10659000A016B701A601CE0101960E94E41561EC98
:1065A00075E0CE0101960E94431620E030E040E104
:1065B00051E4C701B601E9D620E030E040EA50E4FA
:1065C0000E94353B20E030E040E052E4EAD7AB01E6
:1065D000BC01CE0101960E94B41566EC75E0CE01B7
:1065E00001960E94431663E176E0CE0101960E9477
:1065F0004316B801CE0101960E9414166CEE75E0A8
:10660000CE0101960E944316BE016F5F7F4FCE01FF
:1066100007960E948716CE01079625DDCE010796C4
:106620000E948216CE0101960E9482162C960FB609
:10663000F894DEBF0FBECDBFDF91CF911F910F91B8
:10664000FF90EF90DF90CF900895CF92DF92EF927E
:10665000FF920F931F93CF93DF93CDB7DEB72C97A5
:106660000FB6F894DEBF0FBECDBF6B017C018A016F
:1066700065E376E0CE0101960E94A016B701A6015F
:10668000CE0101960E94E41561EC75E0CE01019601
:106690000E94431620E030E040E151E4C701B6011A
:1066A00074D620E030E040EA50E4DFD720E030E06C
:1066B00040E052E476D7AB01BC01CE0101960E94C6
:1066C000B41566EC75E0CE0101960E9443166AE5AA
:1066D00076E0CE0101960E944316B801CE010196E4
:1066E0000E9414166CEE75E0CE0101960E944316CE
:1066F000BE016F5F7F4FCE0107960E948716CE01C5
:106700000796B1DCCE0107960E948216CE01019653
:106710000E9482162C960FB6F894DEBF0FBECDBF36
:10672000DF91CF911F910F91FF90EF90DF90CF906D
:106730000895CF92DF92EF92FF920F931F93CF9322
:10674000DF93CDB7DEB72C970FB6F894DEBF0FBE40
:10675000CDBF6B017C018A016CE776E0CE0101962A
:106760000E94A016B701A601CE0101960E94E41571
:1067700061EC75E0CE0101960E94431620E030E006
:1067800040E151E4C701B60100D620E030E040EA24
:1067900050E46BD720E030E040E052E402D7AB0198
:1067A000BC01CE0101960E94B41566EC75E0CE01E5
:1067B00001960E94431661EA76E0CE0101960E949E
:1067C0004316B801CE0101960E9414166CEE75E0D6
:1067D000CE0101960E944316BE016F5F7F4FCE012E
:1067E00007960E948716CE0107963DDCCE010796DC
:1067F0000E948216CE0101960E9482162C960FB638
:10680000F894DEBF0FBECDBFDF91CF911F910F91E6
:10681000FF90EF90DF90CF900895CF93DF93E2ED5C
:10682000F8E01382128288EE93E0A0E0B0E0848367
:106830009583A683B78320E132E03183208325EC62
:1068400030E03587248724EC30E03787268720EC3A
:1068500030E0318B208B21EC30E0338B228B22EC2B
:1068600030E0358B248B26EC30E0378B268B118E75
:10687000128E138E148ECAEBD9E01B821A828C837F
:106880009D83AE83BF8382E292E099838883EFE6A3
:10689000F9E080E580831182E1E7F9E01582168254
:1068A0001186138682E090E0A0E0B0E084879587AF
:1068B000A687B78713A215A614A686E492E093A72D
:1068C00082A717A6AAE0BAE013961C921E9212970E
:1068D00020EF30E015963C932E93149780E491E0DE
:1068E00017969C938E93169719963C932E93189710
:1068F0001B969C938E931A9755961C9255971D96AE
:106900001C921E921C971F961C921E921E9781E04D
:1069100054968C9354972FEF3FEF53963C932E93BE
:10692000529751963C932E93509756968C93569728
:1069300057961C92579759961C921E925897D59627
:106940001C92D597D6961C92D697D8961C921E92DA
:10695000D797DA961C921E92D99781E390968C93E2
:10696000909780E391968C9391978FEF92968C936A
:10697000929725E43AE05B963C932E935A97939630
:106980008C93939794968C93949795968C939597D4
:106990005C961D921D921D921C925F979B961C9275
:1069A0001E929A97D2961C92D29797961C921E92FC
:1069B0009697D0961C92D09799961C921E92989773
:1069C000D1961C92D197E9E8F3E0E491F0E0EE0F64
:1069D000FF1FE15CFC4F859194919D969C938E9353
:1069E0009C97E9E2F3E0E491D496EC93D497EAE83B
:1069F000F3E0E491F0E0EE0FFF1FE15CFC4F8591C6
:106A000094919F969C938E939E97EAE2F3E0E49193
:106A1000D396EC93D3978EE592E08D939C93E1E02F
:106A2000FAE0138212828EE892E091838083D6830B
:106A3000C583E8EFF9E01382128291838083D683C5
:106A4000C583EFEEF9E01382128291838083D683AF
:106A5000C583E6EEF9E01382128291838083D683A8
:106A6000C583A2EDB9E08AE312968C9312978BE36B
:106A700014968C9314978EE113968C9313978FE151
:106A800015968C9315978DE491E017969C938E93B1
:106A90001697E8E7F3E0E491F0E0EE0FFF1FE15C0A
:106AA000FC4F8591949119969C938E931897E3E9E6
:106AB000F3E0E491F0E0EE0FFF1FE15CFC4F859105
:106AC00094911B969C938E931A97E4E9F3E0E491DA
:106AD000F0E0EE0FFF1FE15CFC4F859194911D9655
:106AE0009C938E931C97E7E7F3E0E491F0E0EE0FC0
:106AF000FF1FE15CFC4F859194911F969C938E93B0
:106B00001E97E8E1F3E0E4915096EC935097E3E3AD
:106B1000F3E0E4915296EC935297E4E3F3E0E491CE
:106B20005196EC935197E7E1F3E0E4915396EC939F
:106B300053978AE090E08D939C9362E975E08CEC2A
:106B400099E00E94A01662E975E086EC99E0DF9179
:106B5000CF910C94A016CF93DF93CDB7DEB7629799
:106B60000FB6F894DEBF0FBECDBF789484B58260B7
:106B700084BD84B5816084BD85B5826085BD85B5E1
:106B8000816085BD80916E00816080936E0010925F
:106B900081008091810082608093810080918100DA
:106BA000816080938100809180008160809380006B
:106BB0008091B10084608093B1008091B0008160C9
:106BC0008093B000809191008260809391008091C9
:106BD000910081608093910080919000816080930A
:106BE00090008091A10082608093A1008091A1001B
:106BF00081608093A1008091A00081608093A000BB
:106C00008091210182608093210180912101816026
:106C100080932101809120018160809320018091E7
:106C20007A00846080937A0080917A0082608093F9
:106C30007A0080917A00816080937A0080917A0056
:106C4000806880937A001092C1000E94E70680E677
:106C5000C82E8AEED82EE12CF12C80918C0A81115D
:106C600010927A0082ED98E00E944A1318161906D5
:106C70000CF052C062E975E0CE0101960E94A016A8
:106C80000E94F30E97FD0CC08F83188641E050E000
:106C9000BE01695F7F4FCE0101960E948715F0CF3C
:106CA00063E975E0CE0107960E94A0164D815E81D2
:106CB00069817A81CE0107960E948715811104C0EF
:106CC000CE0107960E945116BE01695F7F4FCE012B
:106CD0000D960E948716CE0107960E948216CE015D
:106CE00001960E94821689899A899C012150310956
:106CF00040E050E0BE01635F7F4FCE0101960E94ED
:106D0000B416CE010196AFD9CE0101960E9482162B
:106D1000CE010D960E9482160E941215A7019601BF
:106D20000ED4683B7B408105910540F40E94CC0461
:106D300064EF71E080E090E00E94DA140E94E713B3
:106D40008CCF86EC99E00E9482168CEC99E00C9432
:106D50008216EF920F931F93CF93DF93E80147FDC5
:106D600002C034E001C034E1E42F440FFF0BF7FF11
:106D700003C0F195E195F109E32E022F2E2FAE010C
:106D80002AD0CE01DF91CF911F910F91EF900895FE
:106D9000BB274A3031F4992322F4BDE290958195C6
:106DA0009F4F01C0BB27FB015527AA27880F991FBA
:106DB000AA1FA41710F0A41B83955051B9F7A05D2A
:106DC000AA3308F0A95DA193009779F7B111B193A7
:106DD0001192CB0165C24F925F926F927F929F9208
:106DE000AF92BF92CF92DF92EF92FF920F931F93D9
:106DF000CF93DF93CDB7DEB729970FB6F894DEBFF8
:106E00000FBECDBF6A01122FB02E2BE3201720F04A
:106E1000FF24F394F00E02C0BCE3FB2E0F2D27E0FD
:106E2000AE014F5F5F4F64D1AC018981982F99709B
:106E3000913031F0E1FC06C0E0FE06C090E205C0F2
:106E40009DE203C09BE201C090E0EE2DE07183FF64
:106E50003CC0911102C083E001C084E0811718F4A6
:106E6000212F281B01C020E0E1110BC0F601822F69
:106E700030E2882319F031938150FBCFC20ED11C30
:106E800020E0992329F0D6019C93F60131966F01F9
:106E9000C6010396E2FE0AC03EE4D6013C9341E4FB
:106EA00011964C93119712963C9306C03EE6F6015C
:106EB000308341E641833283FC01322F40E23323A9
:106EC00009F442C041933150FACF82FF44C091117E
:106ED00002C083E001C084E0811718F4212F281B31
:106EE00001C020E0E1110BC0F601822F30E28823BF
:106EF00019F031938150FBCFC20ED11C20E09923B1
:106F000029F0D6019C93F60131966F01C6010396D4
:106F1000E2FE0BC039E4D6013C933EE411963C936B
:106F2000119736E412963C9307C039E6F601308398
:106F30003EE6318336E63283FC01322F40E23323D2
:106F400019F041933150FBCFFC01E20FF11D10828B
:106F50008EEF9FEFB7C0F1E0911101C0F0E06F2F0D
:106F600070E01416150624F49A012F5F3F4F02C0FB
:106F700021E030E0260F371FBB2029F06B2D70E099
:106F80006F5F7F4F02C060E070E0260F371F612FF8
:106F900070E0261737071CF4121B212F01C020E0D8
:106FA0003E2D387159F4D601322F60E2332319F0A7
:106FB0006D933150FBCFC20ED11C20E0FF2331F086
:106FC000D6019C93B6016F5F7F4F6B01E1110BC03F
:106FD000F601922F30E3992319F031939150FBCFB2
:106FE000C20ED11C20E09F2D940F3A81782F707132
:106FF000A72E84FF03C0313309F49150191624F4ED
:10700000993018F098E001C091E0E42F852F57FFE8
:1070100002C0E0E080E06E2F782FE0E0F0E0AEE22A
:107020009A2E3A01691A71082A01461A570A0B2D3D
:1070300010E01195019511096F3F8FEF780729F442
:10704000D6019C92C60101966C014617570784F041
:10705000661677066CF47F01E40CF51CA1E0B0E045
:10706000AC0FBD1FEA0EFB1ED7011196BC9002C0EB
:1070700090E3B92E615071093196C60101967C01E9
:107080006017710724F0D601BC926C01D5CF64174C
:10709000750741F4363320F4353321F4A11002C0D2
:1070A00081E3B82EF601B082F701822F90E28823A7
:1070B00019F091938150FBCFF701E20FF11D10827F
:1070C00080E090E029960FB6F894DEBF0FBECDBFEA
:1070D000DF91CF911F910F91FF90EF90DF90CF90B4
:1070E000BF90AF909F907F906F905F904F9008956A
:1070F000283008F027E03327DA01990F311D87FD8A
:10710000916000966105710539F432602E5F3D9300
:1071100030E32A95E1F708959F3F30F080387105FC
:10712000610509F03C5F3C5F3D93913008F0806859
:10713000911DDF93CF931F930F93FF92EF92192F1F
:10714000987F9695E92F96959695E90FFF27EE592A
:10715000FE4F99273327EE24FF24A701E70105906E
:107160000894079428F4360FE71EF81E491F511D96
:10717000660F771F881F991F0694A1F70590079443
:1071800028F4E70EF81E491F561FC11D770F881FF0
:10719000991F661F0694A1F70590079428F4F80E2E
:1071A000491F561FC71FD11D880F991F661F771FC4
:1071B0000694A1F70590079420F4490F561FC71FA6
:1071C000D81F990F661F771F881F0694A9F784910F
:1071D0001095177041F0D695C79557954795F79438
:1071E000E7941A95C1F7E8E0F1E0689415901591DD
:1071F00035916591959105907FE27395E118F10ABB
:10720000430B560BC90BD009C0F7E10CF11E431F0D
:10721000561FC91FD01D7EF4703311F48A95E6CF36
:10722000E894015030F0080F0AF40027021708F420
:10723000202F2395022F7A3328F079E37D932A9526
:10724000E9F710C07D932A9589F60694979567957E
:10725000379517951794E118F10A430B560BC90B94
:10726000D00998F023957E9173957A3308F070E3F6
:107270007C932013B8F77E9170617D9330F08395F5
:1072800071E37D9370E32A95E1F71124EF90FF906D
:107290000F911F91CF91DF91992787FD90950895C8
:1072A000DC01FC01672F71917723E1F7329704C06D
:1072B0007C916D9370836291AE17BF07C8F30895F8
:1072C00040D008F481E00895E89409C097FB3EF4AB
:1072D00090958095709561957F4F8F4F9F4F992323
:1072E000A9F0F92F96E9BB279395F69587957795A1
:1072F0006795B795F111F8CFFAF4BB0F11F460FF61
:107300001BC06F5F7F4F8F4F9F4F16C0882311F0B8
:1073100096E911C0772321F09EE8872F762F05C0CC
:10732000662371F096E8862F70E060E02AF09A9567
:10733000660F771F881FDAF7880F9695879597F95C
:107340000895990F0008550FAA0BE0E8FEEF1616F6
:107350001706E807F907C0F012161306E407F50749
:1073600098F0621B730B840B950B39F40A2661F0BD
:10737000232B242B252B21F408950A2609F4A14060
:10738000A6958FEF811D811D08950BD078C069D01F
:1073900028F06ED018F0952309F05AC05FC0112470
:1073A000A2C07ED0A0F3959FD1F3950F50E0551F5A
:1073B000629FF001729FBB27F00DB11D639FAA274A
:1073C000F00DB11DAA1F649F6627B00DA11D661F99
:1073D000829F2227B00DA11D621F739FB00DA11DBA
:1073E000621F839FA00D611D221F749F3327A00D74
:1073F000611D231F849F600D211D822F762F6A2F10
:1074000011249F5750408AF0E1F088234AF0EE0F94
:10741000FF1FBB1F661F771F881F91505040A9F7A1
:107420009E3F510570F014C05EC05F3FECF3983E84
:10743000DCF3869577956795B795F795E7959F5F08
:10744000C1F7FE2B880F911D9695879597F90895A2
:1074500097F99F6780E870E060E008959FEF80EC07
:10746000089500240A9416161706180609060895AA
:1074700000240A9412161306140605060895092E10
:107480000394000C11F4882352F0BB0F40F4BF2B7F
:1074900011F460FF04C06F5F7F4F8F4F9F4F0895BF
:1074A00057FD9058440F551F59F05F3F71F04795B5
:1074B000880F97FB991F61F09F3F79F0879508959A
:1074C000121613061406551FF2CF4695F1DF08C0B9
:1074D000161617061806991FF1CF869571056105D6
:1074E00008940895E894BB2766277727CB0197F97E
:1074F0000895052E97FB16F400940FD057FD05D084
:107500001ED007FC02D046F408C050954095309537
:1075100021953F4F4F4F5F4F0895909580957095FF
:1075200061957F4F8F4F9F4F08952BD0A59F900D52
:10753000B49F900DA49F800D911D11240895A1E288
:107540001A2EAA1BBB1BFD010DC0AA1FBB1FEE1FDD
:10755000FF1FA217B307E407F50720F0A21BB30B28
:10756000E40BF50B661F771F881F991F1A9469F7A4
:1075700060957095809590959B01AC01BD01CF0100
:107580000895A29FB001B39FC001A39F700D811DFC
:107590001124911DB29F700D811D1124911D08951C
:1075A0005058BB27AA270ED06ACF5BDF30F060DFD0
:1075B00020F031F49F3F11F41EF450CF0EF4E0950B
:1075C000E7FB46CFE92F6CDF80F3BA17620773073A
:1075D0008407950718F071F49EF584CF0EF4E095BA
:1075E0000B2EBA2FA02D0B01B90190010C01CA017D
:1075F000A0011124FF27591B99F0593F50F4503E28
:1076000068F11A16F040A22F232F342F4427585F19
:10761000F3CF469537952795A795F0405395C9F731
:107620007EF41F16BA0B620B730B840BBAF09150E9
:10763000A1F0FF0FBB1F661F771F881FC2F70EC088
:10764000BA0F621F731F841F48F48795779567955B
:10765000B795F7959E3F08F0B3CF9395880F08F044
:107660009927EE0F9795879508950CD008CF00DFE6
:1076700040F0F7DE30F021F45F3F19F0E9CE511110
:1076800032CFECCE0DDF98F39923C9F35523B1F334
:10769000951B550BBB27AA2762177307840738F081
:1076A0009F5F5F4F220F331F441FAA1FA9F333D0E0
:1076B0000E2E3AF0E0E830D091505040E695001C94
:1076C000CAF729D0FE2F27D0660F771F881FBB1F50
:1076D000261737074807AB07B0E809F0BB0B802D2A
:1076E000BF01FF2793585F4F2AF09E3F510568F076
:1076F000AFCEF9CE5F3FECF3983EDCF386957795FD
:107700006795B795F7959F5FC9F7880F911D969577
:10771000879597F90895E1E0660F771F881FBB1FD3
:10772000621773078407BA0720F0621B730B840B80
:10773000BA0BEE1F88F7E0950895AA1BBB1B51E119
:1077400007C0AA1FBB1FA617B70710F0A61BB70BD1
:10775000881F991F5A95A9F780959095BC01CD0176
:107760000895EE0FFF1F881F8BBF0790F691E02D45
:10777000199407DF332312F48A1B9B0B01C001DF2E
:10778000B7FF0895821B930B0895CF93DF93823048
:10779000910510F482E090E0E091060BF091070B68
:1077A00020E030E0C0E0D0E0309711F1408151811D
:1077B00048175907C0F04817590761F4828193812F
:1077C000209719F09B838A832BC09093070B80939B
:1077D000060B26C02115310519F04217530718F47E
:1077E0009A01BE01DF01EF010280F381E02DDCCFC1
:1077F0002115310509F1281B390B2430310590F48E
:1078000012968D919C9113976115710521F0FB01E2
:107810009383828304C09093070B8093060BFD0132
:10782000329644C0FD01E20FF31F819391932250E1
:1078300031092D933C933AC02091040B3091050BF4
:10784000232B41F420910602309107023093050B5F
:107850002093040B2091040230910502211531057B
:1078600041F42DB73EB74091080250910902241B04
:10787000350BE091040BF091050BE217F307A0F430
:107880002E1B3F0B2817390778F0AC014E5F5F4F76
:107890002417350748F04E0F5F1F5093050B409398
:1078A000040B8193919302C0E0E0F0E0CF01DF91FF
:1078B000CF9108950F931F93CF93DF93009709F40F
:1078C0008CC0FC013297138212820091060B10913A
:1078D000070B0115110581F420813181820F931F5F
:1078E0002091040B3091050B2817390779F5F09397
:1078F000050BE093040B71C0D80140E050E0AE17D7
:10790000BF0750F412962D913C911397AD012115AC
:10791000310509F1D901F3CF9D01DA0133832283C7
:1079200060817181860F971F8217930769F4EC01BC
:1079300028813981260F371F2E5F3F4F31832083E7
:107940008A819B8193838283452B29F4F093070BD3
:10795000E093060B42C01396FC93EE931297ED0151
:10796000499159919E01240F351FE217F30771F4D5
:1079700080819181840F951F029611969C938E931E
:107980008281938113969C938E931297E0E0F0E0AE
:10799000D80112968D919C911397009719F0F801D8
:1079A0008C01F6CF8D919C9198012E5F3F4F820FF5
:1079B000931F2091040B3091050B2817390769F4A8
:1079C000309729F41092070B1092060B02C0138215
:1079D00012821093050B0093040BDF91CF911F913E
:1079E0000F9108956F927F928F929F92AF92BF9264
:1079F000CF92DF92EF92FF920F931F93CF93DF937B
:107A0000EC01009781F4CB01DF91CF911F910F9191
:107A1000FF90EF90DF90CF90BF90AF909F908F90AE
:107A20007F906F90B2CEFC01E60FF71F9C012250B1
:107A30003109E217F30708F4A8C0D9010D911C9190
:107A4000119706171707A8F00530110508F49BC019
:107A5000C80104978617970708F495C002501109CA
:107A6000061B170B019311936D937C93CF0122DFBB
:107A70008AC05B01A01AB10A4C01800E911EA09130
:107A8000060BB091070B40E050E0E12CF12C109771
:107A900009F44AC0A815B905D1F56D907C901197ED
:107AA000630182E0C80ED11CCA14DB0480F1A3017B
:107AB0004A195B096A0182E0C80ED11C1296BC907B
:107AC00012971396AC91B5E0CB16D10440F0B28278
:107AD000A38351834083D9016D937C930AC00E5FC9
:107AE0001F4FC301800F911FF90191838083EB2DFC
:107AF000FA2FE114F10431F0D7011396FC93EE93C1
:107B0000129741C0F093070BE093060B3CC08D9198
:107B10009C9111974817590708F4AC017D01129602
:107B20000D90BC91A02DB3CF8091040B9091050BCB
:107B300088159905E1F446175707C8F480910402A7
:107B400090910502009741F48DB79EB740910802CD
:107B500050910902841B950BE817F907B0F4F093D4
:107B6000050BE093040BF901718360830CC0CB011A
:107B70000CDE7C01009749F0A801BE0128D0CE019F
:107B800099DEC70104C0CE0102C080E090E0DF9121
:107B9000CF911F910F91FF90EF90DF90CF90BF900A
:107BA000AF909F908F907F906F90089581E090E0CC
:107BB000F8944FC0FB01DC0104C08D910190801945
:107BC00021F441505040C8F7881B990B0895FB01E0
:107BD000DC0102C001900D9241505040D8F7089549
:107BE000FB01DC018D91019080190110D9F3990BF3
:107BF0000895FB01DC0101900D920020E1F708954A
:107C0000FB01DC014150504048F001900D920020F2
:107C1000C9F701C01D9241505040E0F70895FB01A3
:107C200051915523A9F0BF01DC014D914517411138
:107C3000E1F759F4CD010190002049F04D91401534
:107C40004111C9F3FB014111EFCF81E090E00197B1
:107C5000089514E0C5E9D4E000E005C0802FFE01DE
:107C600080DD2196011DC639D10780E00807B1F7F4
:047C7000F894FFCFB6
:107C7400FFFFFFFF0000080B800000000000000071
:107C84008013EE121913C6134A1328133C13000071
:107C940000002121F220C904C620EA20D620C720F2
:107CA400000000001F14EE12C904C8041F141F149E
:107CB4001F1400000000D528EE12C904C8040000F7
:107CC40000001F14EE12C904C80400000000142CA4
:107CD400EE12C904C804EC196E1A3C1A111EA81934
:107CE4009519E62EC419761F511F5B192119E31843
:107CF400BD2D472DE82CC01FAB1E00000000442200
:107D0400EE12C904C8048022CD235F220D22000094
:107D14000000CD18D019C904BC19AC18A31DAC1DA2
:107D240000010203000102035B20494E464F205D1F
:107D340020536F696C2073656E736F7220312075E8
:107D44006E706C75676765642E005B20494E464F04
:107D5400205D20536F696C2073656E736F722031E0
:107D640020636F6E6E65637465642E005B20494EFC
:107D7400464F205D20536F696C2073656E736F727C
:107D8400203220756E706C75676765642E005B2009
:107D9400494E464F205D20536F696C2073656E73A6
:107DA4006F72203220636F6E6E65637465642E009B
:107DB4005B20494E464F205D20536F696C207365EC
:107DC4006E736F72203320756E706C7567676564AF
:107DD4002E005B20494E464F205D20536F696C2076
:107DE40073656E736F72203320636F6E6E65637498
:107DF40065642E005B20494E464F205D20536F6919
:107E04006C2073656E736F72203420756E706C75A0
:107E1400676765642E005B20494E464F205D205302
:107E24006F696C2073656E736F72203420636F6E9C
:107E34006E65637465642E006762732E626D7000F4
:107E4400206D7300426F6F74696E672047726565B9
:107E54006E686F7573654F532E2E2E7C7C005B46C7
:107E640041494C45445D2053442043617264206E73
:107E74006F7420646574656374656421005B2020FD
:107E84004F4B20205D20456E61626C696E672070E7
:107E94006F776572736176696E6720666561747564
:107EA4007265732E2E2E20202020202020202020BA
:107EB4002020005B20204F4B20205D20456E616216
:107EC4006C6564204C6576656C203120706F776535
:107ED40072736176696E672E005B20204F4B202001
:107EE4005D20456E61626C6564204C6576656C202E
:107EF4003220706F776572736176696E672E005BEE
:107F040020204F4B20205D20456E61626C6564200B
:107F14004C6576656C203320706F7765727361767B
:107F2400696E672E7C5B20494E464F205D20416C74
:107F34006C20706F776572736176696E6720666511
:107F440061747572657320656E61626C65642E0080
:107F54005B20204F4B20205D20536F696C2073659C
:107F64006E736F72203120636F6E6E656374656427
:107F74002E2056657273696F6E3A20005B20204F85
:107F84004B20205D20536F696C2073656E736F7294
:107F9400203220636F6E6E65637465642E205665AF
:107FA4007273696F6E3A20005B20204F4B20205D76
:107FB40020536F696C2073656E736F722033206376
:107FC4006F6E6E65637465642E2056657273696F97
:107FD4006E3A20005B20204F4B20205D20536F69B8
:107FE4006C2073656E736F72203420636F6E6E65E0
:107FF400637465642E2056657273696F6E3A20004F
:108004000D0A0053657269616C3A20005B20204FB1
:108014004B20205D20536F696C2073656E736F7203
:1080240020342074656D70657261747572653A20D0
:108034000020432C200020467C005B20204F4B2056
:10804400205D20536F696C2073656E736F722034EA
:10805400206D6F6973747572653A200025005B208A
:10806400204F4B20205D20536F696C2073656E7325
:108074006F7220332074656D7065726174757265FA
:108084003A20005B20204F4B20205D20536F696C09
:108094002073656E736F722033206D6F697374750E
:1080A40072653A20005B20204F4B20205D20536FE7
:1080B400696C2073656E736F7220322074656D7005
:1080C400657261747572653A20005B20204F4B2005
:1080D400205D20536F696C2073656E736F7220325C
:1080E400206D6F6973747572653A20005B20204FB0
:1080F4004B20205D20536F696C2073656E736F7223
:1081040020312074656D70657261747572653A20F2
:10811400005B20204F4B20205D20536F696C20733F
:10812400656E736F722031206D6F6973747572653B
:048134003A200000ED
:020000023000CC
:10E000000D9489F10D94B2F10D94B2F10D94B2F129
:10E010000D94B2F10D94B2F10D94B2F10D94B2F1F0
:10E020000D94B2F10D94B2F10D94B2F10D94B2F1E0
:10E030000D94B2F10D94B2F10D94B2F10D94B2F1D0
:10E040000D94B2F10D94B2F10D94B2F10D94B2F1C0
:10E050000D94B2F10D94B2F10D94B2F10D94B2F1B0
:10E060000D94B2F10D94B2F10D94B2F10D94B2F1A0
:10E070000D94B2F10D94B2F10D94B2F10D94B2F190
:10E080000D94B2F10D94B2F10D94B2F10D94B2F180
:10E090000D94B2F10D94B2F10D94B2F10D94B2F170
:10E0A0000D94B2F10D94B2F10D94B2F10D94B2F160
:10E0B0000D94B2F10D94B2F10D94B2F10D94B2F150
:10E0C0000D94B2F10D94B2F10D94B2F10D94B2F140
:10E0D0000D94B2F10D94B2F10D94B2F10D94B2F130
:10E0E0000D94B2F141546D656761323536300041AF
:10E0F000726475696E6F206578706C6F72657220DE
:10E1000073746B3530305632206279204D4C530099
:10E11000426F6F746C6F616465723E004875683F52
:10E1200000436F6D70696C6564206F6E203D200048
:10E130004350552054797065202020203D20005FF9
:10E140005F4156525F415243485F5F3D2000415658
:10E1500052204C696243205665723D20004743437C
:10E160002056657273696F6E203D20004350552024
:10E1700049442020202020203D20004C6F7720663D
:10E18000757365202020203D20004869676820665F
:10E190007573652020203D200045787420667573D6
:10E1A00065202020203D20004C6F636B2066757336
:10E1B000652020203D20004D617220203720323024
:10E1C000313300312E362E3800342E332E350056A2
:10E1D00023202020414444522020206F7020636F70
:10E1E00064652020202020696E73747275637469E1
:10E1F0006F6E2061646472202020496E74657272B3
:10E20000757074006E6F20766563746F7200726A49
:10E210006D702020006A6D70200057686174207056
:10E220006F72743A00506F7274206E6F7420737541
:10E2300070706F72746564004D7573742062652030
:10E2400061206C6574746572002000577269747483
:10E25000696E672045450052656164696E672045B7
:10E26000450045452065727220636E743D00504F35
:10E27000525400303D5A65726F2061646472003FF1
:10E280003D43505520737461747300403D454550C3
:10E29000524F4D207465737400423D426C696E6B41
:10E2A000204C454400453D44756D70204545505215
:10E2B0004F4D00463D44756D7020464C415348001B
:10E2C000483D48656C70004C3D4C69737420492F83
:10E2D0004F20506F72747300513D51756974005234
:10E2E0003D44756D702052414D00563D73686F7707
:10E2F00020696E7465727275707420566563746FF0
:10E30000727300593D506F727420626C696E6B00BD
:10E310002A0011241FBECFEFD1E2DEBFCDBF01E046
:10E320000CBF12E0A0E0B2E0EEE1FDEF03E00BBFB6
:10E3300002C007900D92A030B107D9F712E0A0E01B
:10E34000B2E001C01D92AE30B107E1F70F9460F367
:10E350000D948DFE01E20EBF0FEF0DBF11241FBE05
:10E360000D9460F30D9400F020E030E040ED57E0B4
:10E3700005C0FA013197F1F72F5F3F4F2817390792
:10E38000C0F308959C01260F311DC901A0E0B0E043
:10E390002F5F3F4FABBFFC018791882361F08093D3
:10E3A000C6008091C00086FFFCCF8091C0008064D1
:10E3B0008093C000EACF08958DE08093C6008091DD
:10E3C000C00086FFFCCF8091C00080648093C000B5
:10E3D0008AE08093C6008091C00086FFFCCF8091C8
:10E3E000C00080648093C00008950F94C2F10F9420
:10E3F000DCF10895FC019081992359F09093C600B7
:10E400008091C00086FFFCCF8091C0008064809323
:10E41000C0003196992379F70895282F982F929567
:10E420009F70892F805D8A3308F0895F8093C600D2
:10E430008091C00086FFFCCF8091C00080648093F3
:10E44000C000822F8F70982F905D9A3308F0995FEB
:10E450009093C6008091C00086FFFCCF8091C000E1
:10E4600080648093C00008959C01FB01853691056E
:10E470001CF46330710594F0C90164E670E00F94F8
:10E480002EFE605D7F4F6093C6008091C00086FFC6
:10E49000FCCF8091C00080648093C0002B30310598
:10E4A00014F43297B4F0C90164E670E00F942EFEC4
:10E4B0006AE070E00F942EFE605D7F4F6093C600AF
:10E4C0008091C00086FFFCCF8091C0008064809363
:10E4D000C000C9016AE070E00F942EFEC0968093E0
:10E4E000C6008091C00086FFFCCF8091C000806490
:10E4F0008093C00008951F93182F8EE692EE60E07F
:10E500000F94C2F11093C6008091C00086FFFCCF2B
:10E510008091C00080648093C0000F94DCF11F9153
:10E5200008952F923F924F925F926F927F928F92B7
:10E530009F92AF92BF92CF92DF92EF92FF920F9392
:10E540001F93DF93CF93CDB7DEB762970FB6F894E2
:10E55000DEBF0FBECDBF382E622ECA01DB015C01CB
:10E560006D01772420E2222E2E010894411C511CBB
:10E570008BC081E0A81680E0B80681E0C80680E084
:10E58000D80628F0C601AA27BB270F940DF2BB2797
:10E59000AD2D9C2D8B2D0F940DF28A2D0F940DF225
:10E5A0002092C6008091C00086FFFCCF8091C00001
:10E5B00080648093C0009DE29093C6008091C0006B
:10E5C00086FFFCCF8091C00080648093C0002092C1
:10E5D000C6008091C00086FFFCCF8091C00080649F
:10E5E0008093C00019828601750188249924A1E0D6
:10E5F0003A1651F03A1620F0B2E03B1661F409C029
:10E600000BBFF701779007C0C7010F9477FE782EF4
:10E6100002C0F7017080872D0F940DF22092C60082
:10E620008091C00086FFFCCF8091C0008064809301
:10E63000C000872D8052F401EF70F0708F3520F408
:10E64000E40DF51D708204C0E40DF51D8EE280839B
:10E650000894E11CF11C011D111D0894811C911CE2
:10E6600090E18916910409F0C2CF80E190E0A0E02A
:10E67000B0E0A80EB91ECA1EDB1E198AC2010F9493
:10E68000FAF10F94DCF16A94662009F072CF629679
:10E690000FB6F894DEBF0FBECDBFCF91DF911F91B3
:10E6A0000F91FF90EF90DF90CF90BF90AF909F9031
:10E6B0008F907F906F905F904F903F902F90089534
:10E6C0002F923F924F925F926F927F928F929F9282
:10E6D000AF92BF92CF92DF92EF92FF920F931F9370
:10E6E000DF93CF93CDB7DEB7CD53D1400FB6F894BB
:10E6F000DEBF0FBECDBF01E20EBF0FEF0DBF94B75F
:10E70000F894A89514BE80916000886180936000A1
:10E7100010926000789493FF05C0E0910002F091A0
:10E7200001021995279A2F9A8091C00082608093E8
:10E73000C00080E18093C40088E18093C1000000A4
:10E74000EE24FF24870144E0A42EB12CCC24DD2448
:10E7500024C0C5010197F1F70894E11CF11C011DCB
:10E76000111D21E2E2162EE4F20620E0020720E06D
:10E77000120718F031E0C32ED12CC801B70127ECE5
:10E780003BE140E050E00F9441FE611571058105C9
:10E79000910519F485B1805885B98091C00087FD35
:10E7A00003C0C114D104A9F2A6014F5F5F4FC25E3E
:10E7B000DE4F59834883CE51D140C25EDE4F8881FF
:10E7C0009981CE51D140019711F00D9410FEC05D9A
:10E7D000DE4F19821882C053D14060E0C15DDE4F28
:10E7E0001882CF52D14088249924C35DDE4F19820C
:10E7F0001882CD52D140C05EDE4F188219821A8233
:10E800001B82C052D140CE5CDE4F188219821A8220
:10E810001B82C253D140EE24FF2487010BBFF701B6
:10E8200007911691C45CDE4F19830883CC53D14005
:10E830000D940BFEC25EDE4F28813981CE51D1404E
:10E840002130310509F52091C600C25EDE4F1982E4
:10E850001882CE51D14022C02F5F3F4F4F4F5F4FA4
:10E86000213082E138078AE7480780E0580780F0C6
:10E87000C45CDE4FE881F981CC53D140EF5FFF4F9C
:10E8800019F0EE27FF27099420E030E040E050E047
:10E890008091C00087FFE0CF2091C600C35DDE4FAE
:10E8A00048815981CD52D1404F5F5F4FC35DDE4FEC
:10E8B00059834883CD52D140213209F063C64A3092
:10E8C000510508F05FC60894811C911C53E0851621
:10E8D000910409F059C600E010E018C081E280936D
:10E8E000C6008091C00086FFFCCF8091C00080648C
:10E8F0008093C0002F5F3F4F2931310579F70F9486
:10E90000DCF10F5F1F4F0530110519F020E030E0FA
:10E91000E5CF10920A0210920B0210920C02109294
:10E920000D02109206021092070210920802109235
:10E930000902109202021092030210920402109235
:10E9400005028FEE90EE60E00F94F5F180E191EE1C
:10E9500060E00F94C2F18091C00087FFFCCF9091DE
:10E96000C600903608F09F759032B8F09093C600BC
:10E970008091C00086FFFCCF8091C00080648093AE
:10E98000C000A0E2A093C6008091C00086FFFCCF2B
:10E990008091C00080648093C000983409F4D7C18E
:10E9A0009934B8F4923409F459C1933458F490333B
:10E9B00019F1903308F4E3C59F33A1F1903409F0C5
:10E9C000DEC5BDC0953409F470C1963409F0D7C5D1
:10E9D00098C1923509F42BC2933538F49C3409F46C
:10E9E000F5C1913509F0CBC518C2963509F445C279
:10E9F000993509F0C4C567C483E792EE62E00F94CD
:10EA0000F5F110920602109207021092080210927D
:10EA1000090210920A0210920B0210920C0210923C
:10EA20000D0213C18FE792EE62E00F94F5F18FEEC5
:10EA300090EE60E00F94F5F181E291EE60E00F94CA
:10EA4000C2F187EB91EE60E00F94F5F180E391EE77
:10EA500060E00F94C2F184EE90EE60E00F94F5F167
:10EA60008FE391EE60E00F94C2F186E090E061E008
:10EA700070E00F9434F20F94DCF18DE591EE60E0DC
:10EA80000F94C2F189EC91EE60E00F94F5F18EE401
:10EA900091EE60E00F94C2F183EC91EE60E00F9490
:10EAA000F5F18CE691EE60E00F94C2F18EE10F94E7
:10EAB0000DF288E90F940DF281E00F940DF20F949E
:10EAC000DCF18BE791EE60E00F94C2F119E0E0E039
:10EAD000F0E010935700E4918E2F0F940DF20F94F5
:10EAE000DCF18AE891EE60E00F94C2F1E3E0F0E03F
:10EAF00010935700E4918E2F0F940DF20F94DCF1D8
:10EB000089E991EE60E00F94C2F1E2E0F0E0109349
:10EB10005700E4918E2F0F940DF20F94DCF188EAE8
:10EB200091EE60E00F94C2F1E1E0F0E01093570045
:10EB30001491812F0F940DF20F94DCF107CF8BE825
:10EB400092EE62E00F94F5F18BE492EE60E00F94A8
:10EB5000F5F10F94DCF100E010E019C0C8016F2D51
:10EB60000F947FFEFF2031F489E492EE60E00F9471
:10EB7000C2F10BC0F092C6008091C00086FFFCCFAE
:10EB80008091C00080648093C0000F5F1F4FC80158
:10EB900081519F41A0E0B0E0ABBFFC01F790BAE229
:10EBA000FB1621F0E2E000301E07C1F60F94DCF105
:10EBB0000F94DCF187E592EE60E00F94F5F10F948D
:10EBC000DCF1CC24DD2400E010E01EC0C8010F946D
:10EBD00077FEF82E882331F489E492EE60E00F94FA
:10EBE000C2F10BC08093C6008091C00086FFFCCFAD
:10EBF0008091C00080648093C000FE1419F00894D6
:10EC0000C11CD11C0F5F1F4FC80181519F41A0E063
:10EC1000B0E0ABBFFC01E790FAE2EF1621F022E092
:10EC20000030120799F60F94DCF10F94DCF182E6C4
:10EC300092EE60E00F94C2F1C60161E070E00F94C3
:10EC400034F20F94DCF10F94DCF110920202109276
:10EC50000302109204021092050278CE89E992EE26
:10EC600062E00F94F5F1279A2F9A16C02F9880E052
:10EC700090E0E0EDF7E03197F1F7019684369105E9
:10EC8000C1F72F9A80E090E0E0EDF7E03197F1F7DF
:10EC9000019684369105C1F78091C00087FFE6CFC9
:10ECA0008091C00087FFFCCF64C485EA92EE62E0E9
:10ECB0000F94F5F140910202509103026091040219
:10ECC0007091050281E020E10F9491F2809102029F
:10ECD00090910302A0910402B091050280509F4FD1
:10ECE000AF4FBF4F8093020290930302A0930402A0
:10ECF000B093050280509041A040B04008F426CE69
:10ED0000A4CF83EB92EE62E00F94F5F140910602FE
:10ED100050910702609108027091090280E020E1A1
:10ED20000F9491F28091060290910702A09108023F
:10ED3000B091090280509F4FAF4FBF4F80930602A2
:10ED400090930702A0930802B0930902FFCD80ECD4
:10ED500092EE62E00F94F5F183E792EE60E00F949B
:10ED6000F5F18FE792EE60E00F94F5F18BE892EE0B
:10ED700060E00F94F5F189E992EE60E00F94F5F10F
:10ED800085EA92EE60E00F94F5F183EB92EE60E09D
:10ED90000F94F5F180EC92EE60E00F94F5F187ECC2
:10EDA00092EE60E00F94F5F188ED92EE60E00F9442
:10EDB000F5F18FED92EE60E00F94F5F18AEE92EEB0
:10EDC00060E00F94F5F183E093EEBDCD87EC92EE19
:10EDD00062E00F94F5F181E40F947BF282E40F94EA
:10EDE0007BF283E40F947BF284E40F947BF285E45E
:10EDF0000F947BF286E40F947BF287E40F947BF20E
:10EE000088E40F947BF28AE40F947BF28BE40F94F6
:10EE10007BF28CE40F947BF299CD88ED92EE62E068
:10EE20000F94F5F1772473948824992409C48FED05
:10EE300092EE62E00F94F5F140910A0250910B02BC
:10EE400060910C0270910D0282E020E10F9491F22A
:10EE500080910A0290910B02A0910C02B0910D02D8
:10EE600080509F4FAF4FBF4F80930A0290930B0289
:10EE7000A0930C02B0930D0269CD8AEE92EE62E08F
:10EE80000F94F5F184EE90EE60E00F94F5F18FECC5
:10EE900091EE60E00F94F5F1662477244301CC5D98
:10EEA000DE4F19821882C452D140D401C301B695F5
:10EEB000A79597958795CA5DDE4F88839983AA8326
:10EEC000BB83C652D140CC5DDE4FA881B981C4520C
:10EED000D1401196CC5DDE4FB983A883C452D14096
:10EEE000CD0162E070E00F9434F2B0E2B093C6005E
:10EEF0008091C00086FFFCCF8091C0008064809329
:10EF0000C000EDE2E093C6008091C00086FFFCCF18
:10EF10008091C00080648093C000F0E2F093C6004E
:10EF20008091C00086FFFCCF8091C00080648093F8
:10EF3000C000CA5DDE4FE880F9800A811B81C6529D
:10EF4000D140BB27A12F902F8F2D0F940DF2CA5DBA
:10EF5000DE4F8881C652D1400F940DF2B0E2FB2EF5
:10EF6000F092C6008091C00086FFFCCF8091C00067
:10EF700080648093C0000DE30093C6008091C000C0
:10EF800086FFFCCF8091C00080648093C00010E2B7
:10EF90001093C6008091C00086FFFCCF8091C00016
:10EFA00080648093C0008BBEF3012791C65DDE4F65
:10EFB0002883CA52D140A22EBB24CC24DD2408943D
:10EFC000611C711C811C911C8BBEF3018791282E42
:10EFD0003324442455240894611C711C811C911C09
:10EFE0008BBEF3013791C55DDE4F3883CB52D140E4
:10EFF0000894611C711C811C911C8BBEF30147910C
:10F00000C45DDE4F4883CC52D140ADEFEA2EAFEF66
:10F01000FA2EAFEF0A2FAFEF1A2F6E0C7F1C801E57
:10F02000911E142D032DF22CEE24EA0CFB1C0C1D5A
:10F030001D1D0F940DF220E22093C6008091C000A8
:10F0400086FFFCCF8091C00080648093C000C65DC5
:10F05000DE4F8881CA52D1400F940DF230E23093D6
:10F06000C6008091C00086FFFCCF8091C000806404
:10F070008093C000C45DDE4F8881CC52D1400F9494
:10F080000DF240E24093C6008091C00086FFFCCFA5
:10F090008091C00080648093C000C55DDE4F888190
:10F0A000CB52D1400F940DF250E25093C6008091A4
:10F0B000C00086FFFCCF8091C00080648093C000B8
:10F0C0008FEFE8168FEFF80680E0080780E018075A
:10F0D00031F484E092EE60E00F94C2F1DFC0D80119
:10F0E000C7018070907CA070B0708050904CA040A0
:10F0F000B040D1F52FEF3FE340E050E0E222F322B1
:10F1000004231523CA5DDE4FA880B980CA80DB8046
:10F11000C652D140AE0CBF1CC01ED11EAA0CBB1CD7
:10F12000CC1CDD1C8EE092EE60E00F94C2F1BB2798
:10F13000A12F902F8F2D0F940DF28E2D0F940DF285
:10F1400030E23093C6008091C00086FFFCCF8091F2
:10F15000C00080648093C0004EE34093C60080915D
:10F16000C00086FFFCCF87C08EE09EEFA0E0B0E03D
:10F17000E822F9220A231B239CE0E91694E9F90608
:10F1800090E0090790E0190709F088C0C45DDE4FE0
:10F19000A881CC52D140EA2EFF2400E010E0102FCD
:10F1A0000F2DFE2CEE24C55DDE4FB881CB52D14031
:10F1B000EB0EF11C011D111DD601C501817090706F
:10F1C000A070B070DC0199278827E80EF91E0A1F8D
:10F1D0001B1F20EF30E040E050E0A222B322C42207
:10F1E000D52241E1AA0CBB1CCC1CDD1C4A95D1F7F1
:10F1F000EA0CFB1C0C1D1D1D81E090E0A0E0B0E0BE
:10F20000282239224A225B2235E1220C331C441C7D
:10F21000551C3A95D1F7E20CF31C041D151D57013E
:10F220006801AA0CBB1CCC1CDD1C85E192EE60E0E1
:10F230000F94C2F1C801AA27BB270F940DF2BB2778
:10F24000A12F902F8F2D0F940DF28E2D0F940DF274
:10F2500090E29093C6008091C00086FFFCCF809121
:10F26000C00080648093C000AEE3A093C60080918C
:10F27000C00086FFFCCF8091C00080648093C000F6
:10F28000C601AA27BB270F940DF2BB27AD2D9C2DDD
:10F290008B2D0F940DF28A2D0F940DF20F94DCF14B
:10F2A000CC5DDE4FE881F981C452D140F99709F471
:10F2B0004DCBF4E0EF2EF12C012D112D6E0C7F1CA7
:10F2C000801E911EF2CD83E093EE62E00F94F5F183
:10F2D0008AE192EE60E00F94C2F18091C00087FF56
:10F2E000FCCF1091C6001F751093C6008091C0001E
:10F2F00086FFFCCF8091C00080648093C0000F9493
:10F30000DCF1812F81548A3108F036C1163409F4BA
:10F3100095C0173490F4133409F44EC0143430F40B
:10F320001134F1F0123409F01DC130C0143409F465
:10F3300059C0153409F016C16BC01A3409F4C4C0A1
:10F340001B3438F4173409F48FC0183409F00AC19B
:10F35000A1C01B3409F4D2C01C3409F003C1E8C0B9
:10F360008FEF81B90DC082B1809582B980E090E0C5
:10F37000E0EDF7E03197F1F70196883C9105C1F790
:10F380008091C00087FFEFCF12B8EFC08FEF84B934
:10F390000DC085B1809585B980E090E0E0EDF7E0A3
:10F3A0003197F1F70196883C9105C1F78091C00033
:10F3B00087FFEFCF15B8D9C08FEF87B90DC088B1DF
:10F3C000809588B980E090E0E0EDF7E03197F1F7C3
:10F3D0000196883C9105C1F78091C00087FFEFCF6F
:10F3E00018B8C3C08FEF8AB90DC08BB180958BB9A7
:10F3F00080E090E0E0EDF7E03197F1F70196883C8E
:10F400009105C1F78091C00087FFEFCF1BB8ADC059
:10F410008FEF8DB90DC08EB180958EB980E090E0F0
:10F42000E0EDF7E03197F1F70196883C9105C1F7DF
:10F430008091C00087FFEFCF1EB897C08FEF80BBD1
:10F440000DC081B3809581BB80E090E0E0EDF7E0F6
:10F450003197F1F70196883C9105C1F78091C00082
:10F4600087FFEFCF11BA81C08FEF83BB0DC084B38C
:10F47000809584BB80E090E0E0EDF7E03197F1F714
:10F480000196883C9105C1F78091C00087FFEFCFBE
:10F4900014BA6BC08FEF809301010FC080910201FD
:10F4A00080958093020180E090E0E0EDF7E03197F5
:10F4B000F1F70196883C9105C1F78091C00087FF64
:10F4C000EDCF1092020151C08FEF809304010FC065
:10F4D0008091050180958093050180E090E0E0ED4A
:10F4E000F7E03197F1F70196883C9105C1F78091DB
:10F4F000C00087FFEDCF1092050137C08FEF8093DA
:10F5000007010FC08091080180958093080180E079
:10F5100090E0E0EDF7E03197F1F70196883C910536
:10F52000C1F78091C00087FFEDCF109208011DC088
:10F530008FEF80930A010FC080910B01809580931B
:10F540000B0180E090E0E0EDF7E03197F1F70196F4
:10F55000883C9105C1F78091C00087FFEDCF1092E4
:10F560000B0103C085E292EEEEC98091C00087FFD7
:10F57000FCCF8091C600EAC988E392EEE4C98CE131
:10F5800091EEE1C988249924933011F1943028F444
:10F59000913089F09230B8F408C0953061F195301F
:10F5A000F0F0963009F048C043C02B3109F042C951
:10F5B00091E06BE13FC96227C15DDE4F2883CF52E6
:10F5C000D14092E037C9B22FA0E0622793E032C960
:10F5D000822F90E0A82BB92B622794E02BC92E3004
:10F5E00009F039C3622795E0C05DDE4F19821882A9
:10F5F000C053D1401FC9E1E0F0E0EC0FFD1FC05D3A
:10F60000DE4F08811981C053D140E00FF11F2083E4
:10F610000F5F1F4FC05DDE4F19830883C053D14079
:10F6200062270A171B0709F005C9D80196E002C92D
:10F63000261709F010C303C0973009F0FBC87724E0
:10F640009981933109F412C19431C8F4963009F4C8
:10F65000D8C0973050F4923009F406C1933009F4C1
:10F660006DC0913009F059C253C0913109F477C08F
:10F67000923108F0BBC0903109F04FC2F5C098310B
:10F6800009F487C0993150F4953109F4EFC09531F0
:10F6900008F4C6C1963109F040C2C2C19A3109F4DA
:10F6A0006CC09A3108F491C09B3109F45BC09D3164
:10F6B00009F033C29D81903359F48F81882311F46E
:10F6C0009EE11CC0813011F091E018C098E916C08D
:10F6D000892F807591F0903539F4E0E0F0E089E011
:10F6E0008093570094910AC0983539F4E3E0F0E034
:10F6F00089E080935700949101C090E01A821B82A8
:10F700008D818C831D829E831F8227E030E009C299
:10F710001A8288E08B8381E48C8386E58D8382E581
:10F720008E8389E48F8383E5888780E589878FE5E9
:10F730008A8782E38B872BE030E0F3C18A818139AD
:10F7400041F0823941F0803911F48FE005C080E04A
:10F7500003C082E001C08AE01A828B8344C0772410
:10F76000739482C08D81882311F48EE12CC0813086
:10F7700011F081E028C088E926C01A82E1E0F0E0BB
:10F7800089E08093570084918B831C8224E030E0D1
:10F79000C8C18B81803589F48C81883039F4E2E0EE
:10F7A000F0E089E08093570084910DC0E0E0F0E044
:10F7B00089E080935700849106C0E3E0F0E089E09F
:10F7C0008093570084911A82DFCF8D81836C99E0FA
:10F7D000E1E0F0E0082E90935700E89507B600FCB2
:10F7E000FDCF1A821B8223E030E09BC180EC8A832C
:10F7F000CE5CDE4F188219821A821B82C253D1401E
:10F800008EC18A8190E0A0E0B0E0582F44273327D2
:10F8100022278B8190E0A0E0B0E0DC0199278827C7
:10F82000282B392B4A2B5B2B8D8190E0A0E0B0E098
:10F83000282B392B4A2B5B2B8C8190E0A0E0B0E089
:10F84000BA2FA92F982F8827282B392B4A2B5B2BCF
:10F85000220F331F441F551FC05EDE4F288339839C
:10F860004A835B83C052D1401A8259C13A81C95C34
:10F87000DE4F3883C753D140CA5CDE4F1882C6536F
:10F88000D1408B81C82EDD24CA5CDE4F488159816E
:10F89000C653D140C42AD52A933109F082C0CE5C28
:10F8A000DE4F88819981AA81BB81C253D1408050AB
:10F8B000904CA340B04030F583E0CE5CDE4FE88052
:10F8C000F9800A811B81C253D140F70100935B008C
:10F8D00080935700E89507B600FCFDCFCE5CDE4F65
:10F8E000088119812A813B81C253D14000501F4FAA
:10F8F0002F4F3F4FCE5CDE4F088319832A833B8313
:10F90000C253D140C05EDE4F488159816A817B81FC
:10F91000C052D140DE011B9631E08C9111962C91A2
:10F9200011971296C75CDE4F2883C953D140C85C3B
:10F93000DE4F1882C853D14090E0C85CDE4FE881AA
:10F94000F981C853D1408E2B9F2B0C01FA01609393
:10F950005B0030935700E89511244E5F5F4F6F4F67
:10F960007F4F0EEFE02E0FEFF02ECE0CDF1CC114F8
:10F97000D10499F685E0C05EDE4F088119812A81A5
:10F980003B81C052D140F80120935B008093570027
:10F99000E89507B600FCFDCF81E180935700E8951C
:10F9A00035C0C05EDE4F88819981AA81BB81C0527B
:10F9B000D140B695A795979587957C018601ABE0D8
:10F9C000AA2EB12CAC0EBD1E0BC0D5016D915D01F0
:10F9D000C7010F947FFE0894E11CF11C01501040F8
:10F9E0000115110591F7A60160E070E0440F551F65
:10F9F000661F771FC05EDE4FE880F9800A811B8199
:10FA0000C052D1404E0D5F1D601F711F1A82C05E33
:10FA1000DE4F488359836A837B83C052D1407FC0C5
:10FA2000FA80C55CDE4FF882CB53D140C65CDE4F16
:10FA30001882CA53D1408B81C82EDD24C65CDE4FAC
:10FA400008811981CA53D140C02AD12A1A828981DA
:10FA5000BE016D5F7F4F843121F59601C05EDE4FA0
:10FA6000E880F9800A811B81C052D1400BBFF701A9
:10FA700087919691DB018C9311969C936E5F7F4FDB
:10FA8000D801C7010296A11DB11DC05EDE4F88835B
:10FA90009983AA83BB83C052D14022503040F1F6F3
:10FAA00036C0C05EDE4F288139814A815B81C052F9
:10FAB000D1400894C108D108760100E010E0089414
:10FAC000C11CD11C0894E11CF11C011D111DE20E8A
:10FAD000F31E041F151F21BDBB27A52F942F832FB5
:10FAE00082BD2F5F3F4F4F4F5F4FF89A80B5DB01CC
:10FAF0008D93BD012E153F054007510761F7C05E8C
:10FB0000DE4F288339834A835B83C052D1409601FC
:10FB10002D5F3F4FFB01108204C080EC8A8322E0FE
:10FB200030E08BE18093C6008091C00086FFFCCF5F
:10FB30008091C00080648093C000C15DDE4FF88179
:10FB4000CF52D140F093C6008091C00086FFFCCF19
:10FB50008091C00080648093C000432F3093C60022
:10FB60008091C00086FFFCCF8091C00080648093AC
:10FB7000C000922F2093C6008091C00086FFFCCF6A
:10FB80008091C00080648093C0008EE08093C600A6
:10FB90008091C00086FFFCCF8091C000806480937C
:10FBA000C00065E1C15DDE4FE880CF52D1406E25D7
:10FBB00069276427FE01319610C090819093C6009A
:10FBC0008091C00086FFFCCF31968091C000806498
:10FBD0008093C0006927215030402115310569F715
:10FBE0006093C6008091C00086FFFCCF8091C0006A
:10FBF00080648093C00085B1805885B9772081F4F6
:10FC0000C15DDE4F0881CF52D1400F5FC15DDE4F35
:10FC10000883CF52D14090E0A0E0B0E00D941AF4F8
:10FC200027982F9880E090E020ED37E0F901319798
:10FC3000F1F7019684369105C9F700008091C00064
:10FC40008D7F8093C00081E180935700E895EE2777
:10FC5000FF270994FFCF90E00D941AF497FB092E2B
:10FC600007260AD077FD04D02ED006D000201AF443
:10FC7000709561957F4F0895F6F7909581959F4F08
:10FC80000895A1E21A2EAA1BBB1BFD010DC0AA1FDD
:10FC9000BB1FEE1FFF1FA217B307E407F50720F0F5
:10FCA000A21BB30BE40BF50B661F771F881F991F70
:10FCB0001A9469F760957095809590959B01AC01B9
:10FCC000BD01CF010895AA1BBB1B51E107C0AA1FAC
:10FCD000BB1FA617B70710F0A61BB70B881F991FED
:10FCE0005A95A9F780959095BC01CD010895F99991
:10FCF000FECF92BD81BDF89A992780B50895262F31
:10FD0000F999FECF1FBA92BD81BD20BD0FB6F89400
:0EFD1000FA9AF99A0FBE01960895F894FFCF63
:040000033000E000E9
:00000001FF
